S02000006F70656E626C745F6F6C696D65785F73746D3332653430372E737265630B
S3150800000000000220D50A0008A10A0008A30A000871
S31508000010A50A0008A70A0008A90A000800000000A7
S31508000020000000000000000000000000AB0A000805
S31508000030AD0A000800000000AF0A0008B10A00086F
S31508000040250B0008250B0008250B0008250B0008C2
S31508000050250B0008250B0008250B0008250B0008B2
S31508000060250B0008250B0008250B0008250B0008A2
S31508000070250B0008250B0008250B0008250B000892
S31508000080250B0008250B0008250B0008250B000882
S31508000090250B0008250B0008250B0008250B000872
S315080000A0250B0008250B0008250B0008250B000862
S315080000B0250B0008250B0008250B0008250B000852
S315080000C0250B0008250B0008250B0008250B000842
S315080000D0250B0008250B0008250B0008250B000832
S315080000E0250B0008250B0008250B0008250B000822
S315080000F0250B0008250B0008250B0008250B000812
S31508000100250B0008250B0008250B0008250B000801
S31508000110250B0008250B0008250B0008250B0008F1
S31508000120250B0008250B0008250B0008250B0008E1
S31508000130250B0008250B0008250B0008250B0008D1
S31508000140250B0008250B0008250B0008250B0008C1
S31508000150250B0008250B0008250B0008250B0008B1
S31508000160250B0008250B0008250B0008250B0008A1
S31508000170250B0008250B0008250B000800000000C9
S30D08000180250B0008250B0008F9
S3150800018810B5054C237833B9044B13B10448AFF3BB
S3150800019800800123237010BDE00100200000000044
S315080001A85C65000808B5034B1BB103490348AFF360
S315080001B8008008BD00000000E40100205C65000816
S315080001C853B94AB9002908BF00281CBF4FF0FF31A8
S315080001D84FF0FF3000F072B9ADF1080C6DE904CEA6
S315080001E800F006F8DDF804E0DDE9022304B07047FC
S315080001F82DE9F047089E04468846002B4BD18A42CB
S31508000208154667D9B2FA82F24AB1C2F1200701FA4D
S3150800021802F320FA07F7954047EA030894404FEA9D
S31508000228154E230CB8FBFEF71FFA85FC0EFB17883C
S3150800023843EA084307FB0CF1994209D9EB1807F179
S31508000248FF3080F01B81994240F21881023F2B4407
S315080002585B1AA4B2B3FBFEF00EFB103344EA034460
S3150800026800FB0CFCA44509D92C1900F1FF3380F0D2
S315080002780781A44540F2048102382C4440EA074025
S31508000288A4EB0C0400271EB1D4400023C6E900439A
S315080002983946BDE8F0878B4209D9002E00F0EB8075
S315080002A80027C6E9000138463946BDE8F087B3FA9B
S315080002B883F7002F47D18B4202D3824200F2FA8095
S315080002C8841A61EB030301209846002EE0D0C6E99C
S315080002D80048DDE702B9FFDEB2FA82F2002A40F0EA
S315080002E88F80491B4FEA154E1FFA85F80127B1FB7F
S315080002F8FEFC230C0EFB1C1143EA014308FB0CF118
S31508000308994207D9EB180CF1FF3002D2994200F24C
S31508000318CD808446591AA3B2B1FBFEF00EFB101421
S3150800032843EA044408FB00F8A04507D92C1900F14C
S31508000338FF3302D2A04500F2B6801846A4EB08049B
S3150800034840EA0C409FE7C7F1200CBB4022FA0CFE96
S315080003584EEA030E01FA07F420FA0CF521FA0CF313
S315080003684FEA1E482543B3FBF8F92C0C08FB19334A
S315080003781FFA8EFA44EA034309FB0AF49C4202FA76
S3150800038807F200FA07F10BD91EEB030309F1FF3050
S3150800039880F087809C4240F28480A9F10209734460
S315080003A81B1BADB2B3FBF8F008FB103345EA034450
S315080003B800FB0AFAA24508D91EEB040400F1FF332C
S315080003C86BD2A24569D90238744440EA0940A0FBB1
S315080003D80289A4EB0A044C45C2464B4654D351D06D
S315080003E8002E69D0B1EB0A0564EB030404FA0CFC89
S315080003F8FD40FC404CEA0505C6E90054002747E7D6
S31508000408C2F1200320FA03F7954001FA02F021FA0F
S3150800041803F34FEA154E3843010CB3FBFEF71FFAF0
S3150800042885F80EFB173341EA034107FB08F38B42AD
S3150800043804FA02F407D9691807F1FF3C2FD28B4250
S315080004482DD9023F2944CB1A81B2B3FBFEF00EFB25
S31508000458103341EA034100FB08F38B4207D96918B0
S3150800046800F1FF3C17D28B4215D902382944C91A1C
S3150800047840EA07473BE73746304609E70746E7E6CF
S315080004881846FBE64145ABD2B8EB020A69EB0E0201
S3150800049801381346A4E76046E9E7184695E767462C
S315080004A8D1E781467CE702382C4447E7ACF1020CD1
S315080004B82B442FE7384608E73746E9E6704700BF72
S315080004C808B503F087FA08BD08B503F093FA08BD1E
S315080004D808B5054B1B6913F0010F01D0002008BDAC
S315080004E800F0D2F80120FAE70000024008B56420B7
S315080004F800F09AF808BD08B500F09CF808BD000099
S3150800050800B5C7B04FF48C720021684606F00CF89F
S315080005186946094805F080FE40B9009B53B19DF825
S31508000528083013F0100F02D1012000E0002047B070
S315080005385DF804FB0020FAE7846500080048704760
S315080005488465000808B50748002380F828320A2277
S31508000558054905F0C7FA18B9024B012283F828227B
S3150800056808BD00BFFC0100207465000810B50D4BD6
S3150800057893F82832012B10D003F0D8F900F1640457
S31508000588094B1B6813F0400F03D103F0CFF9A042BB
S31508000598F6D9064805F06AFE10BD024805F06EFD54
S315080005A8EAE700BFFC010020001401408465000842
S315080005B808B5054B93F82832012B00D008BD024828
S315080005C805F05CFDFAE700BFFC01002038B50546D2
S315080005D8134B93F82832012B0CD1114905F0CEFE9E
S315080005E8002807DA0E48002380F8283205F046FD69
S315080005F800E001352B788BB10A4A536003F096F967
S3150800060800F10A04074B1B6813F0800FF1D103F0B9
S3150800061881FA03F08BF9A042F4D9EAE738BD00BF9E
S31508000628FC01002000140140014B1880704700BFE8
S315080006382804002008B503F079F90F4B1B6898427F
S3150800064810D30E4B1B7873B90C4B01221A700C4B3E
S315080006584FF000529A6103F069F90A4B1B8818444F
S31508000668054B186008BD054B00221A70044B4FF459
S3150800067800529A61EFE700BF2C0400202A040020E4
S315080006880008024028040020024B4FF400529A61E1
S31508000698704700BF0008024030B58DB000240894A2
S315080006A809940A940B94204B1A6B42F004021A63B5
S315080006B81A6B02F004020592059A1A6B42F0800238
S315080006C81A631A6B02F080020492049A1A6B42F0B3
S315080006D801021A631A6B02F001020392039A1A6B53
S315080006E842F008021A631A6B02F008020292029A8A
S315080006F81A6B42F002021A631B6B03F0020301939A
S31508000708019B0A484FF40053836106930125079510
S3150800071806A901F083FE069507940A9406A90448D3
S3150800072801F07CFE0DB030BD0038024000080240DA
S315080007380000024010B590B0002409940A940B945E
S315080007480C940D940E940F94069407941D4B5A6CAA
S3150800075842F020025A645A6C02F020020292029A67
S315080007681A6B42F004021A631B6B03F00403019325
S31508000778019BC023039302230493032305930823A9
S31508000788089303A9104801F049FE4FF4E133099389
S315080007980A940B940C940C230D930E940F940B4CFB
S315080007A809A9204602F022FB236923F49043236112
S315080007B8636923F02A036361E36843F40053E3603B
S315080007C810B010BD0038024000080240001401406D
S315080007D808B52A4A136823F00F0343F00503136084
S315080007E8264B1B6803F00F03052BF9D1244A136817
S315080007F843F48043136002F5E432136843F4803304
S315080008081360204B1B6813F4003FFAD01D4B5A6837
S315080008181D4911401D4A0A435A605A6822F4403253
S315080008285A601A6842F080721A60164B1B6813F0F1
S31508000838007FFAD0134B9A6822F0F0029A609A68F9
S3150800084822F4E05242F4A0529A609A6822F460426E
S3150800085842F400429A609A6822F0030242F00202C1
S315080008689A60084B9B6803F00C03082BF9D10848D3
S3150800087802F086FB002000F069F908BD003C02403A
S3150800088800700040003802400080BFFF0C5440004A
S31508000898007A030A08B500F07FF9FFF799FFFFF712
S315080008A8FBFEFFF747FFFFF70BFEFFF70DFEFCE71A
S315080008B882B0002100910B4B5A6C42F480425A646C
S315080008C85A6C02F480420092009A01911A6C42F01E
S315080008D880521A641B6C03F080530193019B02B083
S315080008E8704700BF0038024000B589B0002303935B
S315080008F8049305930693079302681A4B9A4202D003
S3150800090809B05DF804FB0022009203F5E833196C78
S3150800091841F080611964196C01F0806100910099B1
S315080009280192196C41F000711964196C01F0007193
S315080009380191019902921A6B42F002021A631B6B23
S3150800094803F002030293029B602303930223049392
S31508000958032306930923079303A9034800F01CFEFB
S31508000968CEE700BF0068004000040240F0B589B031
S315080009780023039304930593069307930268204B71
S315080009889A4201D009B0F0BD0024009403F58633D5
S315080009985A6C42F400625A645A6C02F40062009275
S315080009A8009A01941A6B42F004021A631A6B02F051
S315080009B804020192019A02941A6B42F008021A6319
S315080009C81B6B03F008030293029B4FF4F853039337
S315080009D802270497032606960C2507950DEB0501AD
S315080009E8084800F0D9FD042303930497059406964E
S315080009F807950DEB0501044800F0CEFDC2E700BFD8
S31508000A08002C014000080240000C024008B501F01D
S31508000A189BFD1B4801F066FC1A4801F063FC1A485E
S31508000A2801F060FC194801F05DFC194B5A6C22F478
S31508000A3800625A641A6C22F080621A641A6C22F0F0
S31508000A4800721A641349CA6822F40052CA605A6CBA
S31508000A5822F020025A641A6B22F004021A631A6BEF
S31508000A6822F002021A631A6B22F001021A631A6C40
S31508000A7822F080521A645A6C22F480425A6408BDDD
S31508000A88000C024000080240000402400000024030
S31508000A9800380240001401407047FEE7FEE7FEE70B
S31508000AA8FEE770477047704708B500F08FF808BD2D
S31508000AB8054BD3F8882042F47002C3F888204FF013
S31508000AC800629A60704700BF00ED00E0DFF834D096
S31508000AD8002103E00C4B5B58435004310B480C4B80
S31508000AE842189A42F6D30B4A02E0002342F8043B1E
S31508000AF8094B9A42F9D3FFF7DBFF05F0D1FCFFF75C
S31508000B08C9FE704700000220286E00080000002071
S31508000B18E0010020E001002048120020FEE700005E
S31508000B2810B5094B4FF0FF321A6200241C625A624C
S31508000B385C621A611C615A615C619A619C61FFF783
S31508000B4865FF204610BD00BF0038024010B50446B0
S31508000B580E4B18784FF47A73B3FBF0F30C4A106807
S31508000B68B0FBF3F000F024FB68B90F2C01D901207B
S31508000B780AE0002221464FF0FF3000F0E5FA054B5F
S31508000B881C60002000E0012010BD00BF0400002002
S31508000B98000000200800002008B50B4B1A6842F42C
S31508000BA800721A601A6842F480621A601A6842F477
S31508000BB880721A60032000F0B5FA0020FFF7C6FF16
S31508000BC8FFF776FE002008BD003C0240034A11687C
S31508000BD8034B1B780B441360704700BF2412002090
S31508000BE80400002038B5044602F0A8FE0546B4F10C
S31508000BF8FF3F02D0044B1B781C4402F09FFE401BA3
S31508000C08A042FAD338BD00BF04000020002800F02F
S31508000C18A18038B5044690F82030D3B12268136805
S31508000C2823F00203136002F089FE054623685A6812
S31508000C3812F0020F10D002F081FE401B0A28F5D9DF
S31508000C48636A43F400336362052384F8203001207D
S31508000C5838BDFFF749FEE1E71A6842F001021A6053
S31508000C6802F06CFE054623685A6812F0010F0DD18A
S31508000C7802F064FE401B0A28F5D9636A43F4003378
S31508000C886362052384F820300120E1E7227E012AE1
S31508000C983DD01A6822F080021A60637E012B3BD089
S31508000CA82268136823F040031360A37E012B39D00A
S31508000CB82268136823F020031360E37E012B37D0DC
S31508000CC82268136843F010031360237F012B35D07D
S31508000CD82268136823F008031360637F012B33D057
S31508000CE82268136823F004031360A368E2681343B1
S31508000CF822691343626913436268013A21681343F8
S31508000D08CB6100206062012384F82030A0E71A68C6
S31508000D1842F080021A60C0E72268136843F040036D
S31508000D281360C2E72268136843F020031360C4E718
S31508000D382268136823F010031360C6E7226813684D
S31508000D4843F008031360C8E72268136843F00403EE
S31508000D581360CAE70120704790F82030013BDBB2E0
S31508000D68012B05D9436A43F480234362012070475F
S31508000D7870B4434BD3F8002242F00102C3F80022AC
S31508000D88D3F8002222F47C52C3F80022D3F80022B2
S31508000D98486A42EA0022C3F800224A6902F01F029A
S31508000DA8012000FA02F2D3F81C42D0430440C3F8E3
S31508000DB81C42CB69B3B9324BD3F80C420440C3F88A
S31508000DC80C42CE688D884C6945EA0645483443F88E
S31508000DD834508E680C884D6944EA0644483503EB56
S31508000DE8C5035C60CB69012B1DD08B69002B32D1FA
S31508000DF8234CD4F804320340C4F804320B698BBB7D
S31508000E081F4BD3F814422040C3F814020B6A012B6F
S31508000E182FD01B4AD2F8003223F00103C2F8003259
S31508000E28002070BC7047164BD3F80C421443C3F81D
S31508000E380C420E688D884C6945EA0645483443F8DD
S31508000E4834508E688C894D6944EA0644483503EB64
S31508000E58C5035C60C9E70A4CD4F804321343C4F8DE
S31508000E680432CBE70648D0F814321343C0F81432D4
S31508000E78CCE70349D1F81C321A43C1F81C22C8E743
S31508000E880064004038B590F82030DBB2012B05D055
S31508000E98436A43F400234362012038BD044602230B
S31508000EA880F820300268136823F00103136002F003
S31508000EB845FD054623685B6813F0010F0DD002F05F
S31508000EC83DFD401B0A28F5D9636A43F4003363627B
S31508000ED8052384F820300120DFE700206062DCE77C
S31508000EE870B490F820400568AD68013CE4B2012C5E
S31508000EF806D9436A43F480234362012070BC7047CD
S31508000F0815F0E05F5BD0C5F30165022D3ED80124D4
S31508000F18AC401C608B68002B3ED10E68CB68046811
S31508000F2843EA465605F118031B01E65003680C699F
S31508000F3805F1180603EB06135C600B7D012B36D00A
S31508000F48D17993791B0443EA0163517943EA01236A
S31508000F581479016823432C012144C1F88C31D178CE
S31508000F6893781B0443EA0163517843EA012311780D
S31508000F7802680B432244C2F88831026818352D01E5
S31508000F88535943F0010353510020B7E7436A43F422
S31508000F98000343620120B1E74C6843EAC403CC68FE
S31508000FA80668234305F1180424013351BEE703688C
S31508000FB803EB0613596841F480715960C0E7436A20
S31508000FC843F400134362012098E790F82030013B68
S31508000FD8DBB2012B01D90020704703689B68890694
S31508000FE831EA030301D0012070470020704730B466
S31508000FF890F82040013CE4B2012C06D9436A43F430
S3150800100880234362012030BC704700296FD10468E9
S31508001018E46814F0030F64D0056801F11B04240181
S315080010282C5904F004049460002C6BD1056801F16E
S315080010381B0424012C59640D1460056801F11B046E
S3150800104824012D5905F00205D560056825446D6803
S3150800105805F00F051561056825446D68C5F307256C
S31508001068956105682C446468240C546104680A016F
S315080010781444D4F8B8411C7004681444D4F8B84128
S31508001088C4F307245C7004681444D4F8B841C4F35C
S3150800109807449C7004681444D4F8B841240EDC70DC
S315080010A804681444D4F8BC411C7104681444D4F880
S315080010B8BC41C4F307245C7104681444D4F8BC41E1
S315080010C8C4F307449C7104682244D2F8BC21120E62
S315080010D8DA71F9B90268D36843F02003D3600020AF
S315080010E891E7436A43F40013436201208BE70468D7
S315080010F8246914F0030F8FD1436A43F4001343623B
S31508001108012080E7056801F11B0424012C59E4082D
S31508001118546092E70268136943F0200313610020BC
S3150800112871E70000074AD36823F4E0631B041B0C25
S31508001138000200F4E060184340F0BF6040F4003055
S31508001148D060704700ED00E030B4174BDB68C3F396
S315080011580223C3F10704042C28BF04241D1D062DE9
S3150800116818D9033B4FF0FF3505FA04F421EA0401C0
S31508001178994005FA03F322EA0303194300280BDB0F
S315080011880901C9B200F1604000F5614080F8001312
S3150800119830BC70470023E5E700F00F000901C9B223
S315080011A8024B1954F4E700BF00ED00E014ED00E027
S315080011B80138B0F1807F0AD2064B5860064AF021FA
S315080011C882F823100020986007221A6070470120C9
S315080011D8704700BF10E000E000ED00E010B40A49CF
S315080011E80C6924F440740C610C6944F440740C616D
S315080011F80C6944F001040C610260BFF36F8F436009
S315080012085DF8044B704700BF003C0240074B1A695B
S3150800121822F440721A611A6942F400721A611A694C
S3150800122842F001021A610160704700BF003C0240A3
S31508001238074B1A6922F440721A611A6942F48072D5
S315080012481A611A6942F001021A610180704700BFE3
S31508001258003C0240064B1A6922F440721A611A6960
S315080012681A611A6942F001021A610170704700BFD3
S31508001278003C0240204BDB6813F0100F07D01F4ACA
S31508001288D36943F01003D3611B4B1022DA601A4B5B
S31508001298DB6813F0200F07D0184AD36943F0080310
S315080012A8D361154B2022DA60134BDB6813F0400F25
S315080012B807D0124AD36943F00403D3610E4B402280
S315080012C8DA600D4BDB6813F0800F07D00B4AD36939
S315080012D843F00203D361084B8022DA60064BDB68C9
S315080012E813F0020F07D0054AD36943F02003D361E8
S315080012F8014B0222DA607047003C0240281200209F
S31508001308094B1B69002B01DB00207047064B074A6F
S315080013185A6002F188325A601B69002B01DB0020EB
S3150800132870470120704700BF003C0240230167450B
S31508001338034A136943F0004313610020704700BF4E
S31508001348003C024038B50446154B0022DA6102F023
S31508001358F5FA0546134BDB6813F4803F0AD0B4F157
S31508001368FF3FF7D0CCB102F0E9FA401BA042F1D909
S3150800137803200DE00B4BDB6813F0010F02D0094B75
S315080013880122DA60074BDB6813F0F20F01D100205F
S3150800139838BDFFF76FFF0120FAE70320F8E700BF1B
S315080013A828120020003C0240F8B51D4C247E012C6A
S315080013B834D01F4616460D460446194B01221A769E
S315080013C84CF25030FFF7BEFF014698B9BCB1012C64
S315080013D81AD0022C1DD032463B462846FFF7FEFE99
S315080013E84CF25030FFF7AEFF01460E4A136923F058
S315080013F8010313610A4B00221A760846F8BDF1B2B2
S315080014082846FFF727FFEBE7B1B22846FFF710FF94
S31508001418E6E731462846FFF7F9FEE1E70221ECE759
S3150800142828120020003C0240074B1A6922F4407231
S315080014381A611A6942F004021A611A6942EA002016
S3150800144840F4803018617047003C024010B449B136
S31508001458012921D0022902D04FF4407403E04FF441
S31508001468007400E000240E4B196921F440711961D3
S315080014781A6922431A611A6922F0F8021A611A6966
S3150800148842EAC00040F0020018611A6942F4803244
S315080014981A615DF8044B70474FF48074E3E700BFA0
S315080014A8003C0240164B1B6813F4007F10D0144BFF
S315080014B81A6822F400721A601A6842F400621A60FE
S315080014C81A6822F400621A601A6842F400721A60EE
S315080014D80B4B1B6813F4806F10D0094B1A6822F45B
S315080014E880621A601A6842F480521A601A6822F4EE
S315080014F880521A601A6842F480621A60704700BF00
S31508001508003C0240F8B5224B1B7E012B3ED00E4606
S3150800151804461F4B01221A764CF25030FFF712FF89
S31508001528074670BB4FF0FF3333602368012B16D08C
S31508001538A568E368A2681344AB4220D9217C2846EB
S31508001548FFF784FF4CF25030FFF7FCFE114A136987
S3150800155823F0FA031361074680B90135E9E761689C
S31508001568207CFFF761FF4CF25030FFF7EBFE074689
S31508001578084A136923F00403136100E03560FFF78E
S3150800158891FF034B00221A763846F8BD0227FBE777
S3150800159828120020003C024000230F2B00F2D780B7
S315080015A8F0B583B039E0072200E00022AA403A43A2
S315080015B80234674D45F82420664A1468F24302EA5D
S315080015C804054F6817F4803F01D046EA0405614CC4
S315080015D82560646802EA04054F6817F4003F01D0DD
S315080015E846EA04055B4C6560A46802EA04054F6888
S315080015F817F4801F01D046EA0405564CA560E4682E
S3150800160822404D6815F4001F01D046EA0402514CE1
S31508001618E26001330F2B00F2988001229A400C6889
S3150800162804EA0206B242F4D14C68651E012D03D9B4
S31508001638112C01D0122C12D185685F000324BC40F6
S3150800164825EA0405CC68BC402C438460456825EA2D
S3150800165802054C68C4F300129A402A434260C468DB
S315080016685F000322BA40D24314408D68BD40254323
S31508001678C5604C68022C01D0122C13D1DD08083538
S3150800168850F825E003F007044FEA840C0F2404FAFF
S315080016980CF42EEA040E0C6904FA0CF444EA0E0457
S315080016A840F82540046822404C6804F00304BC400E
S315080016B8224302604A6812F0805FAAD0002201928B
S315080016C8254A546C44F480445464526C02F48042AB
S315080016D80192019A9C08A51C1D4A52F8257003F028
S315080016E8030295000F22AA4027EA02071B4A9042DE
S315080016F83FF45BAF02F5806290421AD002F5806229
S31508001708904218D002F58062904216D002F580629F
S31508001718904214D002F58062904212D002F5806297
S31508001728904210D002F5806290423FF43CAF0822FE
S315080017383CE701223AE7022238E7032236E7042281
S3150800174834E7052232E7062230E703B0F0BD7047D2
S3150800175800380140003C01400038024000000240C1
S3150800176870B582B0044600230193006801F058FA60
S31508001778064610B1304602B070BD206801F063FA1B
S3150800178838B90123A364A36C012B0BD03546304620
S3150800179814E00023A364206801F042FA0028F2D076
S315080017A80646E7E70021206801F064FA0028EDD02C
S315080017B84FF08056DEE7019B01330193019A4FF6F5
S315080017C8FE739A4213D895B90021206801F052FA97
S315080017D8D8B91249206801F065FA0546B8B9002152
S315080017E8206801F060F8C30FE5D01D46E3E7019AC3
S315080017F84FF6FE739A420DD810F0804F02D1002397
S315080018086364B7E701236364B4E70646B2E74FF0B3
S315080018188056AFE74FF08076ACE700BF000010C1EE
S315080018282DE9F04188B004460F4602F087F80646C7
S315080018380023009301930821206801F047F905461B
S3150800184818B1284608B0BDE8F081216D090420685A
S3150800185801F010FA05460028F3D14FF0FF3302933A
S31508001868082303933023049302230593002306933E
S315080018780123079302A9206801F016F9206801F0E8
S3150800188842FA05460028DCD1804605E002F056F8FB
S31508001898801BB0F1FF3F43D02068426B40F22A43D1
S315080018A81A420AD1436B13F4001FEFD000F0D2FF97
S315080018B84DF8280008F10108E8E7436B13F0080F0C
S315080018C825D1436B13F0020F24D1436B13F0200F75
S315080018D823D140F23A538363019A130203F47F0330
S315080018E843EA0263110A01F47F410B4343EA126390
S315080018F83B60009A130203F47F0343EA0263110A62
S3150800190801F47F410B4343EA12637B6099E7082594
S31508001918856396E70225856393E72025856390E71F
S315080019284FF000458DE710B582B0044600210091B6
S315080019380191006800F0B7FF10F0007F16D16946DC
S315080019482046FFF76DFF034690B9019B13F4802FD5
S3150800195811D0216D0904206801F08CF9034638B9BD
S315080019680221206801F0B7F9034601E04FF4006345
S31508001978184602B010BD4FF08063F9E710B582B07B
S315080019880446002100910191006800F08CFF10F0D0
S31508001998007F16D169462046FFF742FF034690B9ED
S315080019A8019B13F4803F11D0216D0904206801F0CA
S315080019B861F9034638B90021206801F08CF9034615
S315080019C801E04FF40063184602B010BD4FF080637B
S315080019D8F9E770B581B10D460446016D090400683A
S315080019E801F0EBF9064608B1304670BD00212068BB
S315080019F800F059FF2860F7E74FF00066F4E70000A3
S31508001A082DE9F04786B004460D4690461E4601F075
S31508001A1895FF6DB1074694F83430DBB2012B0DD02B
S31508001A28A36B43F00053A363012006B0BDE8F08713
S31508001A38A36B43F00063A3630120F6E70023A363BF
S31508001A4808EB0603E26D93421BD8032384F8343067
S31508001A5823680022DA62636C012B01D04FEA482812
S31508001A684FF40071206801F031F8034678B122680E
S31508001A787C499163A06B1843A063012084F834005D
S31508001A88D3E7A36B43F00073A3630120CDE74FF0B8
S31508001A98FF3300937302019390230293022303935F
S31508001AA800230493012305936946206800F0FCFF88
S31508001AB8012E0CD9022323634146206801F036F823
S31508001AC88246BAF1000F0AD1DDF804902FE0012307
S31508001AD823634146206801F011F88246F1E7236836
S31508001AE8604A9A63A36B43EA0A03A363012084F84E
S31508001AF834000023236398E7206800F0ABFE2870BB
S31508001B08C0F307236B70C0F30743AB70000EE87089
S31508001B180435A9F1040908F10108B8F1070FEBD94A
S31508001B2801F00CFFC01B0E9B98420FD273B12068B8
S31508001B38426B40F22A331A4216D1436B13F4004F0C
S31508001B48EED0B9F1000FEBD0D046E6E72368454A50
S31508001B589A63A36B43F00043A363012384F83430E4
S31508001B6800232363032060E7436B13F4807F08D0C0
S31508001B78012E06D9636C032B03D001F01FF8002841
S31508001B8837D123685A6B12F0080F3ED15A6B12F0F8
S31508001B98020F46D15A6B12F0200F4ED12068436BBC
S31508001BA813F4001F55D0B9F1000F52D000F052FEB9
S31508001BB82870C0F307236B70C0F30743AB70000E99
S31508001BC8E8700435A9F1040901F0B8FEC01B0E9B9C
S31508001BD8984201D2002BE1D12368224A9A63A36B63
S31508001BE843F00043A363012084F8340000232363E9
S31508001BF81BE723681B499963A36B0343A363012067
S31508001C0884F83400002323630FE7164A9A63A36B04
S31508001C1843F00803A363012084F8340000232363F0
S31508001C2803E7104A9A63A36B43F00203A3630120F0
S31508001C3884F8340000232363F7E60A4A9A63A36BF9
S31508001C4843F02003A363012084F8340000232363A8
S31508001C58EBE640F23A538363012384F834300020D4
S31508001C68E3E600BFFF0540002DE9F04788B00446C3
S31508001C780D4690461E4601F061FE6DB1074694F87A
S31508001C883430DBB2012B0DD0A36B43F00053A363AA
S31508001C98012008B0BDE8F087A36B43F00063A3638F
S31508001CA80120F6E70023A36308EB0603E26D9342D7
S31508001CB81BD8032384F8343023680022DA62636C5D
S31508001CC8012B01D04FEA48284FF40071206800F02C
S31508001CD8FDFE034678B1226867499163A06B1843ED
S31508001CE8A063012084F83400D3E7A36B43F000739C
S31508001CF8A3630120CDE74FF0FF33029373020393E2
S31508001D08902304930023059306930123079302A9B6
S31508001D18206800F0C9FE012E0CD92023236341460A
S31508001D28206800F033FF8246BAF1000F0AD1DDF8C1
S31508001D380C9033E0102323634146206800F00EFF19
S31508001D488246F1E723684C4A9A63A36B43EA0A0377
S31508001D58A363012084F834000023236399E72B78CA
S31508001D686A7843EA0223AA7843EA0243EA7843EA06
S31508001D78026308A941F81C3D0435A9F1040920683D
S31508001D8800F06BFD08F10108B8F1070FE7D901F073
S31508001D98D5FDC01B109B98420FD273B12068426BC1
S31508001DA840F21A331A4216D1436B13F4804FEED019
S31508001DB8B9F1000FEBD0D046E6E723682E4A9A63B6
S31508001DC8A36B43EA0A03A363012384F83430002388
S31508001DD8236303205DE7436B13F4807F07D0012E46
S31508001DE805D9636C032B02D000F0E8FEC0B9236856
S31508001DF85A6B12F0080F1FD15A6B12F0020F27D12F
S31508001E085A6B12F0100F2FD01B4A9A63A36B43F034
S31508001E181003A363012084F834000023236338E7FA
S31508001E28236815499963A36B0343A363012084F8C0
S31508001E383400002323632CE70F4A9A63A36B43F005
S31508001E480803A363012084F834000023236320E7EA
S31508001E58094A9A63A36B43F00203A363012084F833
S31508001E6834000023236314E740F23A529A630123A5
S31508001E7884F8343000200CE7FF05400010B4436EA0
S31508001E889B0F0B70436EC3F383634B7090F86730F0
S31508001E9803F003038B7090F86630CB7090F86530C2
S31508001EA80B7190F864304B71836E1B0DCB80B0F8BC
S31508001EB86A3003F00F030B72836EC3F3C0334B7299
S31508001EC8836EC3F380338B72836EC3F34033CB724E
S31508001ED8836EC3F300330B7300234B73436C002BD9
S31508001EE840F08880826E40F6FC7303EA8203C26E6D
S31508001EF843EA92730B61C36EC3F3C2630B7590F81A
S31508001F086F3003F007034B75C36EC3F342538B75E3
S31508001F18C36EC3F38243CB75C36EC3F3C2330B7662
S31508001F280B69013343650A7E02F00702023203FA97
S31508001F3802F242650B7A03F00F040123A340836576
S31508001F485B0A03FB02F3C3654FF400730366C36EAB
S31508001F58C3F380334B76C36EC3F3C6138B76C36E4F
S31508001F6803F07F03CB76036FDB0F0B77036FC3F39F
S31508001F7841734B77036FC3F382638B77036FC3F39E
S31508001F888353CB77036FC3F3405381F8203000237C
S31508001F9881F82130B0F8722002F0010281F8222077
S31508001FA8026FC2F3C03281F82320026FC2F380326F
S31508001FB881F82420026FC2F3403281F82520026F87
S31508001FC8C2F3003281F82620026FC2F3812281F813
S31508001FD82720026FC2F3012281F82820026FC2F374
S31508001FE8460281F82920012281F82A2018465DF838
S31508001FF8044B7047012B0BD003680E4A9A63836B10
S3150800200843F080538363012380F834301846EEE79B
S31508002018836E1B0403F47C13B0F86E2013430B611C
S315080020280B6901339B024365C3654FF400738365E7
S3150800203803668CE7FF05400070B590B00446012397
S31508002048ADF81230006800F015FC00286CD0636CF7
S31508002058032B45D1636C032B5DD1636C032B1DD011
S31508002068BDF8121021650904206800F079FE0546B6
S3150800207800285BD10021206800F015FC6066042161
S31508002088206800F010FCA0660821206800F00BFC08
S31508002098E0660C21206800F006FC20670421206809
S315080020A800F001FC000DE06405A92046FFF7E6FEEE
S315080020B800283ED1226D12040023206800F098FDFE
S315080020C8054698BB234653F8106B93E807008DE836
S315080020D80700043494E80E00304600F09FFB25E01C
S315080020E8206800F028FE054600BB0021206800F09D
S315080020F8DAFB60670421206800F0D5FBA067082191
S31508002108206800F0D0FBE0670C21206800F0CBFBC4
S31508002118C4F880009EE70DF11201206800F035FE2C
S315080021280546002899D001E04FF08065284610B08A
S3150800213870BD4FF08055F9E770B58AB0054600239B
S3150800214804930593069307930893762309930AAB92
S3150800215813E907008DE8070004AB0ECB286800F0E2
S315080021685DFB18B1012420460AB070BD0446104E1E
S3150800217800233360286800F075FB0123336028467E
S31508002188FFF7EEFA034630B1012485F83440A86B08
S315080021981843A863E7E72846FFF74EFF03460028D3
S315080021A8E1D0012485F83440A86B1843A863DAE718
S315080021B8A0802542C0B110B5044690F834307BB1EA
S315080021C8032384F834302046FFF7B6FF034670B970
S315080021D80022A2632263012284F83420184610BD1F
S315080021E80377FEF7C3FBEBE701231846704701237D
S315080021F8F4E7436C0B60836C4B60C36C8B60036DB0
S31508002208CB60436D0B61836D4B61C36D8B61036E48
S31508002218CB6100207047000030B58BB004460D46E8
S31508002228032380F83430436C032B1CD0B1F5805F48
S3150800223808D0B1F5006F0AD079B1836B43F0006313
S31508002248836314E0836B43F0805383630FE0FFF7DF
S315080022586AFBA36B1843A06309E0FFF78FFBA36B20
S315080022681843A06303E0836B43F080538363A36B2F
S315080022783BB12368104A9A63012084F834000BB0EE
S3150800228830BD63680493A3680593E36806930795C6
S3150800229863690893A36909930AAB13E907008DE8EC
S315080022A8070004AB0ECB206800F0B8FA012384F8BF
S315080022B834300020E3E700BFFF05400010B582B0C0
S315080022C8044602A9002341F8043DFFF782FB18B12A
S315080022D80346A06B1843A0630198C0F3432002B0D5
S315080022E810BD0000444B984219D0444B984222D05E
S315080022F8434B98422BD0434B984234D0424B984292
S315080023083DD0424B984246D0414B98424FD0414B1C
S31508002318984258D0404B984261D00120704703F53F
S3150800232860531A6942F001021A611A6922F0010219
S315080023381A610020704703F550531A6942F00202E1
S315080023481A611A6922F002021A610020704703F519
S3150800235840531A6942F004021A611A6922F0040203
S315080023681A610020704703F530531A6942F00802CB
S315080023781A611A6922F008021A610020704703F5E3
S3150800238820531A6942F010021A611A6922F01002DB
S315080023981A610020704703F510531A6942F02002A3
S315080023A81A611A6922F020021A610020704703F59B
S315080023B800531A6942F040021A611A6922F040026B
S315080023C81A610020704703F5E0531A6942F0800243
S315080023D81A611A6922F080021A610020704703F50B
S315080023E8C0531A6942F480721A611A6922F4807213
S315080023F81A610020704700BF00000240000402402E
S3150800240800080240000C0240001002400014024076
S3150800241800180240001C024000200240F0B40A6876
S3150800242892FAA2F2B2FA82F22DE00E69C46893FA19
S31508002438A3F5B5FA85F56D00032707FA05F524EA25
S31508002448050493FAA3F5B5FA85F56D0006FA05F5B8
S315080024582C43C4604C68022C3FD04C68056893FA34
S31508002468A3F6B6FA86F67600032707FA06F625EAE5
S31508002478060593FAA3F3B3FA83F35B0004FA03F3A6
S315080024882B43036001320B6833FA02F459D001244E
S3150800249894402340F6D04C68013C012CC5D88E6878
S315080024A8846893FAA3F5B5FA85F56D00032707FA44
S315080024B805F524EA050493FAA3F5B5FA85F56D003A
S315080024C806FA05F52C438460CD68446824EA0304B3
S315080024D803FB05F52C434460A7E793FAA3F4B4FA7B
S315080024E884F4072C15D84E69046A93FAA3F5B5FA45
S315080024F885F5AD000F2707FA05F524EA050493FACA
S31508002508A3F5B5FA85F5AD0006FA05F52C43046278
S31508002518A3E74D69466A1C0A94FAA4F7B7FA87F737
S31508002528BF004FF00F0C0CFA07F726EA070694FACD
S31508002538A4F4B4FA84F4A40005FA04F4344344620F
S315080025488BE70020F0BC704782B0234A136843F033
S3150800255801031360204B1B6813F0020FFAD01E4BB9
S3150800256800229A601A680192019A22F0867222F469
S3150800257880320192019A22F080620192019A1A60C9
S315080025881A6822F0F80242F080021A60124B1B6899
S3150800259813F0007FFAD1104B104A5A60104AC3F854
S315080025A88420DA6822F4F852DA60DA6822F40052EB
S315080025B8DA60DA6842F41F02DA60DA6842F400126E
S315080025C8DA605A6F22F001025A675A6F42F080722F
S315080025D85A67002002B070470038024010300024BD
S315080025E800300020034B9B68C3F30313024AD35CED
S315080025F8D840704700380240A4650008034B9B681A
S31508002608C3F38223024AD35CD84070470038024095
S31508002618B4650008034B9B68C3F34233024AD35C8C
S31508002628D840704700380240B46500080F4B5B680D
S3150800263803F4800323B90E4B082803D000207047FB
S315080026480C4BF9E7094A506800F03F00B3FBF0F372
S315080026585068C0F3881000FB03F05368C3F30143BE
S3150800266801335B00B0FBF3F0704700BF0038024047
S315080026780024F400001BB70008B5084B9B6803F054
S315080026880C03042B07D0082B01D0054808BD0820E1
S31508002698FFF7CCFFFAE70348F8E700BF003802401F
S315080026A80024F400001BB70010B50446FFF7E4FF42
S315080026B82060FFF797FF6060FFF7A0FFA0606068DB
S315080026C8FFF7A8FFE06010BD0B4B1B680B4AA2FB7F
S315080026D803235A0A41F2883303FB02F35A1E43B10D
S315080026E8416B134611F0800FF8D0C5238363002089
S315080026F870474FF00040704700000020D34D621025
S31508002708154B1B68154AA2FB03235A0A41F288335C
S3150800271803FB02F35A1EDBB1416B134611F0450F52
S31508002728F8D011F4006FF5D1436B13F0040F07D1F5
S31508002738436B13F0010F07D1C52383630020704745
S315080027480423836318467047012383631846704732
S315080027584FF00040704700BF00000020D34D6210BC
S31508002768114B1B68114AA2FB03235A0A41F2883304
S3150800277803FB02F35A1E9BB1416B134611F0450F32
S31508002788F8D011F4006FF5D1436B13F0040F03D199
S31508002798C52383630020704704238363184670475C
S315080027A84FF00040704700BF00000020D34D62106C
S315080027B8184B1B68184AA2FB03235A0A41F28833A6
S315080027C803FB02F35A1EFBB1416B134611F0450F82
S315080027D8F8D011F4006FF5D1436B13F0040F0BD141
S315080027E8436B13F0010F0BD1436B13F0400F0ED058
S315080027F84023836300207047042383631846704781
S3150800280801238363184670474FF00040704700203D
S31508002818704700BF00000020D34D621084B010B482
S3150800282802AC84E80E000B46039A1343049A134332
S31508002838059A1343069A1343079A1343426822F4E0
S31508002848FD4222F07F021343436000205DF8044BE3
S3150800285804B07047D0F8800070470B68C0F880301D
S315080028680020704708B5032303600220FEF7BAF96B
S31508002878002008BD006800F0030070470B688360F5
S315080028884B688A681343CA6813430A691343C268BC
S3150800289822F47F6222F00F021343C36000207047B8
S315080028A80069C0B2704714304058704738B5524B63
S315080028B81B68524CA4FB03435B0A02FB03F2531E34
S315080028C8002A60D0446B1A4614F0450FF7D014F462
S315080028D8006FF4D1436B13F0040F07D1436B13F061
S315080028E8010F07D00123836318464EE00423836348
S315080028F818464AE00D460446C5238363FFF7D0FF0A
S31508002908A84201D0012040E000212046FFF7CBFF6E
S315080029183B4B0340D3B300283ADB10F0804F3AD13B
S3150800292810F0005F39D110F0805F38D110F0006FD1
S3150800293838D110F0806F38D110F0807F38D110F474
S31508002948000F38D110F4800F38D110F4001F38D191
S3150800295810F4801F38D110F4802F38D110F4003FB6
S3150800296838D110F4803F38D110F4004F38D110F41C
S31508002978804F38D110F4005F38D110F0080F38D0DE
S315080029884FF4000001E04FF0004038BD0020FCE796
S315080029984FF00070F9E74020F7E78020F5E74FF495
S315080029A88070F2E74FF40070EFE74FF48060ECE7C9
S315080029B84FF40060E9E74FF48050E6E74FF400501B
S315080029C8E3E74FF48040E0E74FF40040DDE74FF4D3
S315080029D80030DAE74FF48020D7E74FF40020D4E731
S315080029E84FF48010D1E74FF40010CEE74FF480007B
S315080029F8CBE74FF48030C8E700000020D34D6210BB
S31508002A0808E0FFFD70B5264B1B68264CA4FB03435C
S31508002A185C0A41F2883303FB04F35C1EB3B3456BC7
S31508002A28234615F0450FF8D015F4006FF5D1436B1A
S31508002A3813F0040F07D1436B13F0010F07D00123D6
S31508002A488363184624E004238363184620E0164661
S31508002A580D460446FFF724FFA84201D0012017E0D7
S31508002A68C523A36300212046FFF71DFF10F4604F16
S31508002A7808D010F4804F0CD110F4004F0CD04FF446
S31508002A88805005E0000C3080002001E04FF000403F
S31508002A9870BD4FF40050FBE74FF48030F8E700BFED
S31508002AA800000020D34D62100B6843624B688362AE
S31508002AB88B68CA6813430A6913434A691343C26A87
S31508002AC822F0F7021343C3620020704730B587B077
S31508002AD80546019110240294402303930023049386
S31508002AE84FF48063059301A9FFF7C8FE41F28832BF
S31508002AF821462846FFF7DAFE07B030BD30B587B05D
S31508002B080546019111240294402303930023049354
S31508002B184FF48063059301A9FFF7B0FE41F28832A6
S31508002B2821462846FFF7C2FE07B030BD30B587B044
S31508002B380546019112240294402303930023049323
S31508002B484FF48063059301A9FFF798FE41F288328E
S31508002B5821462846FFF7AAFE07B030BD30B587B02C
S31508002B6805460191182402944023039300230493ED
S31508002B784FF48063059301A9FFF780FE41F2883276
S31508002B8821462846FFF792FE07B030BD30B587B014
S31508002B9805460191192402944023039300230493BC
S31508002BA84FF48063059301A9FFF768FE41F288325E
S31508002BB821462846FFF77AFE07B030BD30B587B0FC
S31508002BC80546002301930C24029440220392049399
S31508002BD84FF48063059301A9FFF750FE034A21467F
S31508002BE82846FFF763FE07B030BD00BF00E1F505CC
S31508002BF830B587B00546019207240294402303930B
S31508002C08002304934FF48063059301A9FFF736FE62
S31508002C1841F2883221462846FFF748FE07B030BDFC
S31508002C2810B586B0044600230193029303930493D0
S31508002C384FF48063059301A9FFF720FE2046FFF7A6
S31508002C4843FD06B010BD10B586B004464FF4D573DB
S31508002C5801930823029340230393002304934FF414
S31508002C688063059301A9FFF709FE2046FFF7A0FD33
S31508002C7806B010BD30B587B00546019137240294D1
S31508002C8840230393002304934FF48063059301A913
S31508002C98FFF7F4FD41F2883221462846FFF706FE7B
S31508002CA807B030BD10B586B0044641F0004141F47E
S31508002CB88011019129230293402303930023049347
S31508002CC84FF48063059301A9FFF7D8FD2046FFF75F
S31508002CD847FD06B010BD30B587B0054601910624F4
S31508002CE8029440230393002304934FF480630593C7
S31508002CF801A9FFF7C3FD41F2883221462846FFF7A6
S31508002D08D5FD07B030BD30B587B005460023019319
S31508002D18332402944022039204934FF48063059364
S31508002D2801A9FFF7ABFD41F2883221462846FFF78D
S31508002D38BDFD07B030BD10B586B004460023019323
S31508002D4802220292C022039204934FF480630593E9
S31508002D5801A9FFF793FD2046FFF7D2FC06B010BD80
S31508002D6810B586B00446019109230293C02303933C
S31508002D78002304934FF48063059301A9FFF77EFDAA
S31508002D882046FFF7BDFC06B010BD70B586B00546EF
S31508002D980E460023019303240294402203920493C7
S31508002DA84FF48063059301A9FFF768FD324621466B
S31508002DB82846FFF727FE06B070BD30B587B005462A
S31508002DC801910D24029440230393002304934FF49E
S31508002DD88063059301A9FFF751FD41F28832214620
S31508002DE82846FFF763FD07B030BD0000C36813F433
S31508002DF8005F01D0012070472DE9F04B84B00D46DD
S31508002E080446C36823F4164323F00C034A68C968C2
S31508002E180A4329690A43A9690A431343C360AB6885
S31508002E28026922F44052134303616B69426922F42A
S31508002E384072134343616846FFF736FC494B9C4288
S31508002E4810D0494B9C4214D0484B9C4213D0484B4F
S31508002E589C4212D0474B9C4211D0474B9C4210D0FB
S31508002E6801207CE00398002878D02B685BB90120FC
S31508002E7875E00298F7E70298F5E70398F3E70298EA
S31508002E88F1E70298EFE7AA69B2F5004F30D04FF09C
S31508002E980009061849EB090716EB000B47EB090C5E
S31508002EA84FEACC0242EA5B724FEACB0594469A008F
S31508002EB89B0F401949EB0C01FDF782F92F4DA5FB2D
S31508002EC8003149090A0192B2642303FB11031B0165
S31508002ED83233A5FB0313C3F34F1303F0F0010A4477
S31508002EE892B203F00F0313449BB2A360002036E0A6
S31508002EF883464FF0000C06184CEB0C0716EB000837
S31508002F0847EB0C094FEAC90242EA58724FEAC80564
S31508002F1891460021DA1841EB01031BEB05004CEB3F
S31508002F280901FDF74DF9154DA5FB003149090A01B7
S31508002F3892B2642303FB1103DB003233A5FB0313A8
S31508002F48C3F34F13590001F4F8710A4492B203F017
S31508002F58070313449BB2A360002000E0012004B0D5
S31508002F68BDE8F08B001001400044004000480040CE
S31508002F7800140140004C0040005000401F85EB51EA
S31508002F88014B1860704700BF0000002000B583B0E9
S31508002F98009313460A4601460348FEF731FD00B179
S31508002FA8012003B05DF804FBA011002000B583B02A
S31508002FB8009313460A4601460348FEF755FE00B134
S31508002FC8012003B05DF804FBA011002008B50348EA
S31508002FD8FFF774F9043818BF012008BDA0110020AE
S31508002FE808B501460148FFF704F908BDA0110020F5
S31508002FF882B001238DF807309DF8070002B07047A4
S3150800300810B5104B104A1A6000225A609A60DA60A6
S315080030181A615A6103229A61FFF7EAFF012802D06A
S315080030280124204610BD0748FFF7C4F804460028BF
S31508003038F7D14FF400610348FFF7EEF80028F0D0FF
S315080030480124EEE7A0110020002C014008B5064B24
S315080030581B780BB1002008BD034B01221A7000200B
S3150800306800F02AF8F7E700BF3004002008B500206A
S3150800307800F036F808BD08B5002000F035F808BD98
S3150800308808B5002000F040F808BD08B5002000F093
S315080030984BF808BD08B5074B01221A70FFF796FFCB
S315080030A820B9044A137803F0FE031370014B187805
S315080030B808BD00BF0C00002010B50446074B0122C6
S315080030C81A70FFF79DFF10B1044B187810BD2046FB
S315080030D8FFF7E0FF014B1870F6E700BF0C00002069
S315080030E808B5FFF7D7FF08BD08B5084611461A46BA
S315080030F84FF0FF33FFF74AFF20B9FFF767FF0028AD
S31508003108FBD108BD0120FCE708B5084611461A4652
S315080031184FF0FF33FFF74AFF20B9FFF757FF00289C
S31508003128FBD108BD0120FCE7154B1B7813F0010FEE
S3150800313821D110B588B0144603291ED8DFE801F056
S3150800314802050C13002008B010BD6846FFF748FFB3
S31508003158069B23600020F6E76846FFF741FF079BB2
S3150800316823800020EFE76846FFF73AFF079B5B0ACC
S3150800317823600020E7E7032070470420E3E700BF41
S315080031880C00002072B6704762B670472DE9F04108
S3150800319884B004460D46174698466846FFF784FAEB
S315080031A80299164BA3FB01318909002201E0013275
S315080031B8D2B2112A1DD8124B13F8120003EB420398
S315080031C893F801C000EB0C0303FB0443B1FBF3FEC1
S315080031D803FB1E16002EEAD11FFA8EF32B80013B3D
S315080031E89BB2B3F5806FE2D2387088F800C0012028
S315080031F800E0002004B0BDE8F08100BFD34D62109E
S31508003208F865000870B58CB00022ADF82E208DF848
S315080032182D200CAB03F8042D0DF12D020DF12E010E
S315080032284FF4FA70FFF7B2FF002836D01D4C1E4B34
S315080032382360002525766576A5760126E676257720
S315080032486577A560E5609DF82D30013B1B04236171
S315080032589DF82C30013B1B056361BDF82E30636071
S315080032682046FDF7D3FC0E230693079508964CF6D9
S31508003278E042019202954FF6E07203920422049204
S31508003288059509960A930DEB02012046FDF764FD9C
S315080032982046FDF7F7FD0CB070BDB521034800F0D0
S315080032A851FBC3E73404002000680040BC650008E9
S315080032B810B588B040F2E17302930023049305938E
S315080032C8069101AB024602A90B48FDF709FE08B1AB
S315080032D808B010BD00F02AFB00F13204019906482F
S315080032E8FDF773FE0028F3D000F014FC00F01EFB6F
S315080032F8A042F3D9ECE700BF3404002010B588B023
S315080033080C46034601AA00210A48FDF770FE60B973
S31508003318019A40F267639A4201D0002006E0039BAF
S3150800332833B9059B2370012000E0002008B010BDC2
S315080033380020FBE73404002008B5FFF723FF08BD83
S3150800334810B500F001FA00B910BDFDF7C1F800285C
S31508003358FAD000F095FBFDF7E3FB00F0BDFA00F0A4
S31508003368F7F920F0604020F07F00044B986000F0E1
S31508003378EFF94468FFF708FFA047E5E700ED00E026
S3150800338870B508E04D1C461C0B78037000F0C2FBAC
S31508003398304629462246531E9CB2002AF2D170BDF1
S315080033A838B50546002401E00134E4B2092C15D8DD
S315080033B800F0B0FB04EB44029300094AD358AB4229
S315080033C8F2D804EB44029100054A0A4452681344A9
S315080033D8AB42E9D9024B0B44187A00E0FF2038BD06
S315080033E81C66000808B5C1F3080353B903688B427D
S315080033F809D040F8041B4FF40072FFF7C1FF0120FB
S3150800340800E0002008BD0120FCE72DE9F041074649
S31508003418FDF776FF00247F2C14D83E68A30006EB38
S3150800342803083B445D6800F075FB2A4600234146BD
S315080034380220FDF7B9FF38B956F82430AB4209D14E
S315080034480134E8E7012400E00024FDF771FF20466F
S31508003458BDE8F0810024F8E738B50D460C4B9842CC
S3150800346811D004460B4B994207D1094C29462046E8
S31508003478FFF7B8FF48B1204638BDFFF7C6FF002852
S31508003488F4D10024F7E7044CF0E70024F3E700BF7B
S3150800349860060020008000085C0400202DE9F04141
S315080034A806460C4617461D4621F4FF7828F00108FB
S315080034B80368B3F1FF3F07D0336843450BD1336838
S315080034C8E41A3444043415E04146FFF78BFF0346F3
S315080034D80028F1D11FE041463046FFF7BDFF0646F2
S315080034E80028ECD1002316E017F8013B04F8013B45
S315080034F8013D0FD000F00EFB331DE31AB3F5007F2C
S31508003508F2D308F500713046FFF7A6FF064628B13C
S31508003518041DE9E701231846BDE8F0810023FAE708
S3150800352870B586B004460D460023009388420ED827
S315080035380126012C1ED90B2D20D8E6B100230193AC
S315080035480223059301230493FDF7DAFE03E0002618
S31508003558EFE70134E4B2AC4209D800F0DBFA039489
S31508003568694601A8FDF7CEFF0028F2D00026FDF728
S31508003578DFFE00E00026304606B070BD0026FAE7F2
S315080035884FF0FF33024A1360024A1360704700BFC0
S315080035985C0400206006002070B54B1E154C241AE2
S315080035A8A34201D9002070BD16460D460446FFF70A
S315080035B8F7FEFF281AD028190138FFF7F1FEFF2869
S315080035C816D024F4FF7323F001030B4A934206D05E
S315080035D82B46324621460948FFF760FFE3E72B46A4
S315080035E8324621460648FFF759FFDCE70020DAE7A6
S315080035F80020D8E7FFFF0F08008000085C040020B9
S31508003608600600204A1E0E4B1B1A9A4201D9002052
S31508003618704770B50C460546FFF7C2FE06466019A0
S315080036280138FFF7BDFEFF2E06D0FF2806D0014653
S315080036383046FFF775FF70BD0020FCE70020FAE763
S31508003648FFFF0F08104B1B68B3F1FF3F1AD000B5F0
S3150800365883B00D4A536891680B44D1680B441169C5
S315080036680B4451690B4491690B44D26913445B4274
S3150800367802AA42F8043D04210448FFF78DFF03B067
S315080036885DF804FB01207047600600208881000861
S315080036980D4B1B680D4A12681A440D4B1B681344D8
S315080036A80C4A126813440C4A12681A440B4B1B68D6
S315080036B81A440B4B1B6813440A4A1268DA4201D0AB
S315080036C80020704701207047008000080480000821
S315080036D8088000080C80000810800008148000087C
S315080036E8188000088881000808B50D4B1B68B3F1D7
S315080036F8FF3F0BD10B4B1B68B3F1FF3F0DD00948B1
S31508003708FFF783FE034648B1012307E00448FFF79D
S315080037187CFE03460028EDD100E00123184608BDC3
S31508003728600600205C0400200048704700800008F6
S3150800373808B5FFF725FF08BD08B5FFF72DFF08BD33
S3150800374808B5FFF75FFF08BD08B5FFF7A1FF08BD75
S3150800375808B5FFF7E9FF08BD08B5FFF773FF034685
S3150800376808B9184608BDFFF7BFFF0346F9E7000082
S31508003778054B1B6813F0200F04D0034B5B680370D6
S3150800378801207047002070470014014010B5094B06
S31508003798586000F0CBF800F10A04064B1B6813F0D2
S315080037A8800F05D100F0B6F900F0C0F8A042F4D9A8
S315080037B810BD00BF0014014010B588B00C4CE36872
S315080037C823F40053E3604FF4614301930023029303
S315080037D8039304930C2205920693079301A920469E
S315080037E8FFF704FBE36843F40053E36008B010BD31
S315080037F80014014070B506460D46402904D82846E7
S31508003808FFF7C4FF00240BE07B21074800F09AF86D
S31508003818F5E700F07FF9305DFFF7B8FF0134A4B289
S31508003828ABB2A342F5D870BD9466000870B5254BAF
S315080038381C78BCB92448FFF79BFF012801D020460D
S3150800384870BD214B1B78013BDBB23F2BF7D800F044
S315080038586DF81E4B18601E4B00221A70194B012270
S315080038681A70ECE706460D46194B1B7801331648BD
S315080038781844FFF77DFF0446012815D1144B1A781A
S315080038880132D2B21A70104B1B789A4201D0002422
S31508003898D5E710493046FFF773FD0A4B00221A7020
S315080038A80B4B1B782B70CAE700F040F8074B1B68D0
S315080038B86433984203D90024024B1C70BFE70024DE
S315080038C8BDE700BFA508002064080020A808002056
S315080038D8A608002065080020024B00221A605A60D4
S315080038E89A60704710E000E008B5FFF7F5FF054B4A
S315080038F8054A5A6000229A6005211960034B1A6026
S3150800390808BD00BF10E000E03F900200AC080020A8
S31508003918044B1B6813F4803F03D0034A136801332A
S315080039281360704710E000E0AC08002008B5FFF700
S31508003938EFFF014B186808BDAC08002008B5FFF76B
S31508003948F5FF08BD08B500F0E5F8FCE708B500F08E
S31508003958D5F8012806D000F06DF918B10C4B1B787C
S31508003968012B00D008BDFFF7E1FF0A4B1B680A4A7E
S315080039781268134403F5FA739842F3D3044B0022EA
S315080039881A7000F061F90028ECD1FFF7D9FCE9E7CD
S31508003998B4080020B0080020B808002008B5054B70
S315080039A81B78012B00D008BDFFF7C0FF024B186033
S315080039B8F9E700BFB4080020B808002008B5044B8A
S315080039C801221A70FFF7EAFFFFF7C0FF08BD00BF1C
S315080039D8B408002008B5FFF7AFFC00F097F8FFF722
S315080039E883FFFFF7A5FE00F00DF900F00FF8FFF7C3
S315080039F8E5FF08BD08B500F08DF8FFF789FF00F068
S31508003A081DFA00F013F8FFF7A1FF08BD10B500F07E
S31508003A1897FDFFF7F7FB044C01232370FFF7CCFE4D
S31508003A280023237010BD00BF0D00002000B583B029
S31508003A380DF107011048FFF761FC012809D00DF1BF
S31508003A4807010D48FFF7F2FE01280BD003B05DF811
S31508003A5804FB0A4B01221A709DF80710064800F065
S31508003A688FFDECE7054B00221A709DF807100248EF
S31508003A7800F086FDEAE700BFBC0800200D0000201C
S31508003A887047000038B504460D46094B1B78012BCC
S31508003A9805D0074B1B7833B100F06AFD38BDC9B2AB
S31508003AA8FFF706FCF5E7E9B22046FFF7A3FEF3E7BA
S31508003AB80D000020074B1B78022B05D0032B05D0D9
S31508003AC8012B05D04020704700207047002070471A
S31508003AD8082070470D000020074B1B78022B05D0DD
S31508003AE8032B05D0012B05D04020704700207047CE
S31508003AF800207047082070470D00002008B500F020
S31508003B082DFD034600B10123184608BD08B5FCF784
S31508003B18EDFC08BD08B5FCF7EEFC08BD10B4034675
S31508003B2801310D4AA2FB0323DB08F9D100230B70E8
S31508003B38094BA3FB0023DB081A4603EB83035C0047
S31508003B48031B303301F8013D1046002AF0D1084618
S31508003B585DF8044B704700BFCDCCCCCC00F00F0302
S31508003B68092802D903F13700704710B503F1300464
S31508003B7802F0BAFC2044437803F00303022B01D071
S31508003B88E0B210BD203CFBE738B505460C460009EF
S31508003B98FFF7E4FF207005F00F00FFF7DFFF6070FE
S31508003BA80023A370204638BDF8B5074600263546D3
S31508003BB807E0203C10E02D01EDB2AB18DDB2013666
S31508003BC8F6B2012E19D8BC5D02F08EFC2044437863
S31508003BD803F00303022BECD0E3B2A3F13002D2B20E
S31508003BE8162A09D8A3F13A01C9B2062907D9092A12
S31508003BF8E1D9373BDAB2DEE700252846F8BD0025C5
S31508003C08FBE7000008B50022064B1A700649074864
S31508003C1801F03CFF00B908BD77210548FFF792FE79
S31508003C28F9E700BF5C0D0020D466000804090020E7
S31508003C38D8660008034B1B780BB100207047012093
S31508003C48704700BF5C0D002008B5FFF757FF01282D
S31508003C580ED0084B1B780BB1002008BDFCF750FCAA
S31508003C68012801D00020F8E7024B01221A70F4E770
S31508003C780020F2E75C0D002038B50546047802F006
S31508003C8833FC2044437803F00303022B03D0532C58
S31508003C9803D0032038BD203CF9E702F025FC6B78F1
S31508003CA81844427812F0040F09D0312B09D0322B68
S31508003CB809D0332B01D00320ECE70220EAE70320DA
S31508003CC8E8E70020E6E70120E4E770B50646023093
S31508003CD8FFF76AFF054684B204363046FFF764FFE5
S31508003CE80544EDB2013CA4B20236012CF5D8ED43E1
S31508003CF8EDB23046FFF758FFA84201D0002070BD44
S31508003D080120FCE7F8B5044617460E46A1B198B156
S31508003D182046FFF7B1FF0546032800F087802046AE
S31508003D28FFF7D3FF002800F08480012D29D04DB174
S31508003D38022D4DD000257AE040F263213E48FFF770
S31508003D4801FEE5E7A01CFFF72FFF85B2201DFFF748
S31508003D582BFF00023060A01DFFF726FF33681844C2
S31508003D6830600834033D2DB2002F60D00026AE42DD
S31508003D785DDA2046FFF718FFB85502340136B6B2A1
S31508003D88F5E7A01CFFF710FF85B2201DFFF70CFF0B
S31508003D9800043060A01DFFF707FF336803EB002017
S31508003DA8306004F10800FFF7FFFE336818443060F6
S31508003DB80A34043D2DB2002F39D00026AE4236DA31
S31508003DC82046FFF7F1FEB85502340136B6B2F5E7D4
S31508003DD8A01CFFF7E9FE85B2201DFFF7E5FE0006E1
S31508003DE83060A01DFFF7E0FE336803EB0040306043
S31508003DF804F10800FFF7D8FE336803EB00203060AB
S31508003E0804F10A00FFF7D0FE3368184430600C3412
S31508003E18053D2DB25FB10026AE4208DA2046FFF707
S31508003E28C3FEB85502340136B6B2F5E7002528466A
S31508003E38F8BD4FF0FF35FAE7D8660008B54B1B788A
S31508003E48002B00F0F58170B5012B05D0022B30D078
S31508003E58032B00F0208170BDFFF76AFCFCF772FBA4
S31508003E68AD48FCF7B3FBAD48FCF7B0FBFCF766FBBF
S31508003E7801220146AA4801F035FE48B1A54B0022A1
S31508003E881A70A848FCF7A2FB0120FCF791FBE2E7A9
S31508003E98A548FCF79BFBA548FCF798FBA448FCF744
S31508003EA895FBA44B00221A605A609A4B02221A7094
S31508003EB8D1E7A14C04F50C724FF480719F4802F0C3
S31508003EC833FA94F84132002B5DD1A8B19B480022F9
S31508003ED800F5C071FFF716FF0446B0F1FF3F60D042
S31508003EE8002809DD934B5B68002B67D1934BD3F801
S31508003EF88021904B1A6058608F4BD3F84422D3F828
S31508003F083C329A42A7D10021854802F0CBF800280E
S31508003F1840F0A780874B5B6873B38348FCF756FB6A
S31508003F288748FCF753FB874D824C29466068FFF79C
S31508003F38F5FD2846FCF74AFB8348FCF747FB294664
S31508003F48E078FFF721FEA91CA078FFF71DFE291DBA
S31508003F586078FFF719FEA91D2078FFF715FE284691
S31508003F68FCF734FB7948FCF731FB61682068FFF7F2
S31508003F78E7FB002800F082806B48FCF727FB654BB7
S31508003F8803221A7067E7634B00221A706548FCF724
S31508003F981DFB0220FCF70CFB04F50C7002F06EF80A
S31508003FA859E75C4B00221A705E48FCF70FFB0320A2
S31508003FB8FCF7FEFA5A4802F061F84CE75F4AD2F86D
S31508003FC880115C4A12681A44914203D10344594A3B
S31508003FD8536091E75448FCF7F9FA5948FCF7F6FA9A
S31508003FE8584E544D31466868FFF798FD3046FCF739
S31508003FF8EDFA5548FCF7EAFA3146E878FFF7C4FDC2
S31508004008B11CA878FFF7C0FD311D6878FFF7BCFD1D
S31508004018B11D2878FFF7B8FD3046FCF7D7FA4B48A4
S31508004028FCF7D4FA69682868FFF78AFB60B13E4846
S31508004038FCF7CCFA3E48FCF7C9FA404BD3F880217E
S315080040483C4B1A605C6057E7324B00221A703548B9
S31508004058FCF7BCFA0520FCF7ABFA314802F00EF873
S31508004068F9E62C4B00221A702E48FCF7AFFA042002
S31508004078FCF79EFA2A4802F001F8ECE6254B0022DE
S315080040881A702848FCF7A2FA0520FCF791FA244882
S3150800409801F0F4FFDFE6284C04F50C724FF4807142
S315080040A8264802F041F994F84132002B56D160B1FE
S315080040B8224800F5807200F5C071FFF723FE044612
S315080040C8B0F1FF3F58D0002863DC1B4BD3F84422D5
S315080040D8D3F83C329A427FF4BEAE1D48FCF776FA0E
S315080040E8FFF73AFB002800F096800F48FCF76EFAAF
S315080040F81848FCF76BFA0A4801F0C0FF1648FCF79F
S3150800410865FA044B00221A70FCF730FAFFF718F91B
S31508004118A1E600BF5C0D0020086700082C670008A8
S31508004128340B0020546700085C67000864670008B9
S3150800413888670008FC08002004090020600D002094
S31508004148B8670008E40E0020C46700086868000815
S31508004158506800086C68000884680008354B002217
S315080041681A703548FCF732FA0220FCF721FA04F5EA
S315080041780C7001F083FF6EE62E4B00221A702F484A
S31508004188FCF724FA0320FCF713FA2D4801F076FF0A
S3150800419861E62C48FCF71AFA2B4D29462046FFF704
S315080041A8BDFC2846FCF712FA2848FCF70FFA284EF1
S315080041B8294696F88301FFF7E7FCA91C96F88201B9
S315080041C8FFF7E2FC291D96F88101FFF7DDFCA91D1A
S315080041D896F88001FFF7D8FC2846FCF7F7F91D483A
S315080041E8FCF7F4F906F580722146D6F88001FFF740
S315080041F8A3FA18B11848FCF7E9F966E70D4B002247
S315080042081A701648FCF7E2F90620FCF7D1F90C48AB
S3150800421801F034FF1FE6074B00221A700F48FCF717
S31508004228D5F90720FCF7C4F9054801F027FF12E677
S31508004238704700BF5C0D0020E067000804680008A6
S31508004248340B002028680008E40E002038680008A7
S31508004258600D0020686800085C6700085467000855
S31508004268014B00225A707047240F0020034BFE2288
S31508004278DA7018710222A3F844207047240F002028
S3150800428810B5054C00232370FFF7EAFFFF23E370F8
S315080042980123A4F8443010BD240F0020064BFF2242
S315080042A8DA7000221A71597859719A71DA711A7284
S315080042B80622A3F844207047240F002008B50020DA
S315080042C8FFF7D4FF08BD0000074BFF22DA70074A3C
S315080042D89A6400221A715A719A710722C3F807203C
S315080042E80822A3F844207047240F0020B068000865
S315080042F8044BFF22DA7042689A640122A3F8442024
S31508004308704700BF240F002008B53120FFF7AEFF1D
S3150800431808BD000038B5084CFF23E3700025257151
S315080043286571FFF7C7FBA071E571257265720723EA
S31508004338A4F8443038BD00BF240F002038B5FFF76D
S3150800434879FCE8B1FFF78CFF0F4C01252570FF2390
S31508004358E3701023237100236371FFF7ABFBA07189
S31508004368FFF7BAFBE071FFF7B7FBC0F30720207227
S315080043786572A5720823A4F84430FFF7D9F938BD41
S315080043881020FFF773FFFAE7240F002038B5054613
S315080043984478FFF78FFB0138844210DC0A4C6A78A8
S315080043A8A16C201DFEF7ECFFFF23E3706A78A36C67
S315080043B81344A3646B780133A4F8443038BD22202B
S315080043C8FFF754FFFAE700BF240F002038B5044664
S315080043D84578FFF76FFB0138854211DC61680A4D9D
S315080043E8A9646278281DFEF7CBFFFF23EB70627875
S315080043F8AB6C1344AB6463780133A5F8443038BD15
S315080044082220FFF733FFFAE7240F0020F8B5054600
S315080044181746002406E015F8013B1C44E4B2FFF7EA
S3150800442879FB31464E1E0029F5D13C600120F8BDBE
S3150800443810B5084CFF23E370E21D4168A06CFFF72E
S31508004448E5FF207100236371A3710823A4F844309B
S3150800445810BD00BF240F002038B505460D4B9C6CCF
S31508004468FFF728FB6A1C411E2046FFF765F960B16D
S31508004478084CFF23E370FFF71DFB0138A36C0344C0
S31508004488A3640123A4F8443038BD3120FFF7EEFEB3
S31508004498FAE700BF240F002038B504464578FFF729
S315080044A809FB023885420EDC114BFF22DA7001221D
S315080044B8A3F84420617851B9FFF74EF930B931208D
S315080044C8FFF7D4FE02E02220FFF7D0FE38BDA21C73
S315080044D8074B986CFFF730F928B16178044A936C52
S315080044E80B449364F2E73120FFF7C0FEEEE700BFFE
S315080044F8240F002008B54168074B986CFFF720F988
S3150800450830B1054BFF22DA700122A3F8442008BD12
S315080045183120FFF7ABFEFAE7240F002008B5FEF7AF
S315080045280FFF034BFF22DA700122A3F8442008BDC7
S31508004538240F002008B589B2FFF7A4FA08BD0000C1
S31508004548054B00221A709A6483F84320A3F844207E
S315080045589A705A70704700BF240F0020034B1B78C7
S315080045680BB1012070470020704700BF240F0020B8
S31508004578024B002283F84320704700BF240F00200F
S3150800458808B50378FF2B04D0354A1278012A14D0C7
S3150800459808BDFFF7D3FE324B93F84330012B5AD0A8
S315080045A82F4BB3F944100029F2DD1846012380F889
S315080045B843300330FFF7BEFFEAE7C93B352B46D839
S315080045C8DFE803F03345454245453F363C3945451E
S315080045D84545454545454545454545454545454575
S315080045E84545454545454545454545454545241EAD
S315080045F81B2145454527452A2D30FFF7C7FECAE73B
S31508004608FFF7E4FEC7E7FFF773FEC4E7FFF710FFF7
S31508004618C1E7FFF759FEBEE7FFF750FEBBE7FFF70E
S315080046283DFEB8E7FFF72CFEB5E7FFF715FFB2E73B
S31508004638FFF732FFAFE7FFF76DFEACE7FFF75AFF64
S31508004648A9E7FFF76BFFA6E7FFF75EFEA3E72020BB
S31508004658FFF70CFE9FE71020FFF708FEA0E700BF4C
S31508004668240F00204278007840EA02207047C27872
S31508004678837843EA0222437843EA0223007840EA29
S31508004688032070470170090A417070470170C1F329
S3150800469807234370C1F307438370090EC170704737
S315080046A813462AB10A78027001300131013BF9D163
S315080046B8704701700130013AFBD1704730B4451C88
S315080046C8037808781B1A013A04D04C1C2846214658
S315080046D8002BF4D0184630BC704700E00130037848
S315080046E80BB18B42FAD11846704702394369023B27
S315080046F88B4204D94389806A01FB0300704700206E
S31508004708704770B506460D4601F11A00FFF7AAFF6D
S315080047183378032B00D070BD044605F11400FFF763
S31508004728A1FF44EA0040F6E770B506460C4615466A
S3150800473891B204F11A00FFF7A5FF3378032B00D0CE
S3150800474870BD290C04F11400FFF79CFFF8E7000078
S315080047582DE9F04107460E4601F11A00FFF782FFD8
S3150800476860BB357805F03F05013D05EB450305EBCC
S3150800477883054FF00108002404E04FF6FF739842BA
S3150800478821D101340C2C0ED8124B185D3044FFF792
S3150800479869FFB8F1000FF0D0FE2D12D827F81500DA
S315080047A880460135EDE7337813F0400F0DD0FE2D1E
S315080047B80DD8002327F81530012000E00020BDE8B1
S315080047C8F0810020FBE70020F9E70120F7E7002041
S315080047D8F5E700BF386900082DE9F84380460F4613
S315080047E891464B730F23CB7200240C73214607F1AD
S315080047F81A00FFF747FF09F1FF3606EB460306EBF3
S315080048088306254602E001340C2C11D84FF6FF73AF
S315080048189D4202D038F8165001360C4B185D2946C9
S315080048283844FFF72FFF002DEDD14FF6FF75EAE75D
S315080048384FF6FF739D4202D038F816300BB949F087
S31508004848400987F80090BDE8F88300BF3869000872
S3150800485870B582B0054616461C460B22FFF720FFA0
S31508004868052C11D807221DE001320F2A0CD803F0AF
S31508004878010101EB44045B0814F4803FF4D084F486
S31508004888883484F02104EFE73388002BEAD002360F
S315080048980022EAE7531E02A8024402F8081C240963
S315080048A809D01A4604F00F0303F130013929F1D962
S315080048B803F13701EEE77E2102461A4402F8081C7E
S315080048C800E001349C4209D22A5D202AF9D105E084
S315080048D82021621C2955072A08D81446072BF7D819
S315080048E802AA1A4412F8081C0133F2E702B070BD8E
S315080048F801460B220020C30143EA5003087850FA00
S3150800490883F3D8B20131013AF5D17047016809B184
S315080049180A4603E04FF0FF3308E0013213781F2BED
S3150800492801D93A2BF9D13A2B02D0002318467047F9
S3150800493810B44C1C0B78303B092B08D8A24209D175
S315080049485BB90132026018465DF8044B70474FF0B0
S31508004958FF33F8E74FF0FF33F5E74FF0FF33F2E799
S3150800496838B50D4640B1044603682BB11A781AB112
S31508004978D9888288914203D000232B60092038BD44
S315080049885878FEF773FB10F0010FF5D123682B60F2
S315080049980020F4E7F8B5C3780BB90020F8BD04463B
S315080049A8C56A00F1300701232A4639464078FEF7DA
S315080049B867FBA8B90023E370236AEB1AA269934236
S315080049C810D2A678012E09D9A3691D4401232A46BF
S315080049D839466078FEF754FB013EF3E70020DDE729
S315080049E80120DBE70020D9E770B5C36A8B4212D0ED
S315080049F804460D46FFF7CEFF064668B901232A4640
S31508004A0804F130016078FEF736FB10B101264FF045
S31508004A18FF35E56200E00026304670BD10B504464D
S31508004A280023C3704FF0FF33C362FFF7DDFFD8B921
S31508004A3804F22E20FFF716FE4AF65523984215D19A
S31508004A4804F16600FFF713FE20F07F400A4B9842F0
S31508004A580ED004F18200FFF70AFE20F07F40064BCD
S31508004A68984207D1002002E0042000E0032010BD88
S31508004A780020FCE70220FAE7464154002DE9F047F2
S31508004A8884B00F46164600230B60FFF73FFF051E46
S31508004A98C0F24181B54B53F82540002C00F03F8100
S31508004AA83C6006F0FE06237873B16078FEF7DEFAF6
S31508004AB810F0010F08D1002E00F0338110F0040F12
S31508004AC840F03181002027E100232370E8B26070A6
S31508004AD8FEF7BCFA10F0010F40F027811EB110F05E
S31508004AE8040F40F0248100212046FFF797FF02288B
S31508004AF800F0B3800026042800F01B81012800F284
S31508004B081A8104F13B00FFF7ADFDB0F5007F40F0D0
S31508004B18148104F14600FFF7A5FD074620B904F1FC
S31508004B285400FFF7A4FD0746A76194F84020A27031
S31508004B38531EDBB2012B00F2028107FB02F594F83B
S31508004B483D80A4F80A80B8F1000F00F0FA8008F151
S31508004B58FF3318EA030F40F0F68004F14100FFF727
S31508004B6881FD8246208110F00F0F40F0EE8004F197
S31508004B784300FFF777FD814620B904F15000FFF797
S31508004B8876FD814604F13E00FFF76CFD01460028D4
S31508004B9800F0DD80421902EB1A129145C0F0D9805F
S31508004BA8A9EB0203B3FBF8F3002B00F0D48040F618
S31508004BB8F570834269D84FF001094FF6F5708342BC
S31508004BC801D94FF0030903F10208C4F81480E66115
S31508004BD88B1923623244A262B9F1030F58D0BAF18D
S31508004BE8000F00F0BE802B446362B9F1020F60D053
S31508004BF808EB480208F0010303EB520303F2FF131C
S31508004C08B7EB532FC0F0AF804FF0FF332361E36053
S31508004C1880232371B9F1030F4ED084F80090544AC3
S31508004C28138801339BB21380E380002074E00020C8
S31508004C3804AB03EB850343F8100C0135032D0ED896
S31508004C4804F130002B0103F5DF7318440379002BB0
S31508004C58EDD00830FFF70BFDEAE70025EEE700255B
S31508004C680AE031462046FFF7D9FE01287FF643AF0A
S31508004C780135032D3FF63FAF04AB03EB850353F825
S31508004C88106C002EEDD10320F2E74FF0020994E7E5
S31508004C9804F15A00FFF7E6FC00285ED1BAF1000FC6
S31508004CA85DD104F15C00FFF7E2FC60624FEA880315
S31508004CB8A4E74FEA4803A1E704F16000FFF7D2FC2E
S31508004CC80128AAD1711C2046FFF78EFE0028A4D118
S31508004CD80023237104F22E20FFF7C4FC4AF6552355
S31508004CE898429AD104F13000FFF7C1FC214B98424B
S31508004CF893D104F50570FFF7BAFC1F4B98428CD17F
S31508004D0804F50670FFF7B3FC206104F50770FFF792
S31508004D18AEFCE06081E70B2004B0BDE8F0870C2004
S31508004D28FAE70020F8E70A20F6E70320F4E70A205E
S31508004D38F2E70120F0E70D20EEE70D20ECE70D205D
S31508004D48EAE70D20E8E70D20E6E70D20E4E70D2061
S31508004D58E2E70D20E0E70D20DEE70D20DCE70D2071
S31508004D68DAE70D20D8E70D20D6E700BF700F002038
S31508004D78740F00205252614172724161F8B5066893
S31508004D88012952D973698B4251D90C463378022BBB
S31508004D982BD0032B38D0012B01D0012046E001EB9C
S31508004DA85105316A01EB55213046FFF71DFE0028EB
S31508004DB83FD16F1CC5F30805354495F83050316A5C
S31508004DC801EB57213046FFF70FFEA8BBC7F30807C4
S31508004DD83E4496F8300045EA002014F0010F01D049
S31508004DE8000923E0C0F30B0020E0316A01EB142127
S31508004DF83046FFF7F9FD10BB600000F4FF7030304D
S31508004E083044FFF72FFC11E0316A01EBD411304624
S31508004E18FFF7EAFDB0B9A00000F4FE703030304460
S31508004E28FFF725FC20F0704000E00120F8BD0120BE
S31508004E38FCE74FF0FF30F9E74FF0FF30F6E74FF0A1
S31508004E48FF30F3E74FF0FF30F0E72DE9F041076848
S31508004E58B1F5001F3BD206460D4611F01F0F39D192
S31508004E68316184681CB93B78022B00D97C6A94B9ED
S31508004E783B89B3EB551F2FD97B6AB3617461B36954
S31508004E8893B303EB5523B3613037C5F308053D449F
S31508004E98F56100201CE0B7F80A804FEA482845451E
S31508004EA80FD321463046FFF769FF0446B0F1FF3FA6
S31508004EB814D0012814D97B69834213D9A5EB0805B0
S31508004EC8EDE721463846FFF710FCB061D6E7022021
S31508004ED8BDE8F0810220FBE70220F9E70120F7E7A1
S31508004EE80220F5E70220F3E70220F1E72DE9F84367
S31508004EF801297CD943698B427BD916460C46054657
S31508004F080378022B47D0032B57D0012B01D0022751
S31508004F1870E001EB5108016A01EB5821FFF764FDBF
S31508004F280746002866D108F10109C8F3080814F0ED
S31508004F38010423D005EB080393F9303003F00F0377
S31508004F48320102F47F621343DBB2A84488F8303092
S31508004F580123EB70296A01EB59212846FFF744FD1E
S31508004F680746002846D1C9F308094CB1C6F3071203
S31508004F78A94489F830200123EB703BE0F3B2E4E753
S31508004F8805EB090393F9302022F00F02C6F303262E
S31508004F983243D2B2ECE7016A01EB1421FFF724FD8C
S31508004FA8074638BB600000F4FF703030B1B22844B9
S31508004FB8FFF768FB0123EB701CE0016A01EBD411CB
S31508004FC8FFF712FD0746A8B926F07046A40004F4B0
S31508004FD8FE7430342C442046FFF749FB00F0704134
S31508004FE831432046FFF752FB0123EB7002E0022704
S31508004FF800E002273846BDE8F8832DE9F041074660
S315080050080668884631B9F5688DB17369AB420FD819
S3150800501801250DE0FFF7B2FE0346012847D9B0F18E
S31508005028FF3F49D07269824246D8454600E00125C5
S315080050382C460CE021463846FFF7A0FE034670B119
S31508005048012839D0B0F1FF3F36D0AC4233D001340D
S315080050587369A342EED8012D2BD90224EAE74FF04B
S31508005068FF3221463046FFF741FF034610B9B8F12B
S31508005078000F0ED1A3B9F46032697369023B9A42EC
S3150800508801D2013A3261337943F001033371234679
S3150800509812E0224641463046FFF728FF0346E9E76D
S315080050A8012B01D0012307E04FF0FF3304E0012369
S315080050B802E0002300E000231846BDE8F081F8B5B1
S315080050C80E46046801292ED9074611466369B34274
S315080050D82BD95AB14FF0FF322046FFF707FF024691
S315080050E820B123E063692E46AB421FD931463846BC
S315080050F8FFF744FE0546D8B101281BD0B0F1FF3F9B
S315080051081AD0002231462046FFF7F0FE024668B953
S315080051182369B3F1FF3FE5D001332361237943F0CF
S3150800512801032371DEE7022200E002221046F8BDD9
S315080051380022FBE70222F9E70122F7E72DE9F843FF
S31508005148066805698369002B6DD02035B5F5001FFB
S315080051586BD288460446C5F308073FB9013383610D
S31508005168416971B93389B3EB551F06D925613037BB
S315080051783E44E6610020BDE8F883002383610420E5
S31508005188F9E77389013B13EA5523EFD1FFF7F6FDD3
S31508005198814601284BD9B0F1FF3F4AD0736983424B
S315080051A839D8B8F1000F11D061692046FFF725FFF5
S315080051B8814600283FD001283FD0B0F1FF3F3ED0B6
S315080051C83046FFF7E7FB28B10120D4E70023A3619F
S315080051D80420D0E74FF40072002106F13000FFF7EB
S315080051E868FA49463046FFF780FAF0624FF0000839
S315080051F8738998450BD20123F3703046FFF7CAFB2B
S31508005208F8B908F10108F36A0133F362F0E7F36ABB
S31508005218A3EB0803F362C4F8149049463046FFF72F
S3150800522864FAA061A2E70420A5E70420A3E7022000
S31508005238A1E701209FE707209DE702209BE70120B9
S3150800524899E7012097E7F8B504460F46066800214E
S31508005258FFF7FBFD0346C0B9002508E00135BD4246
S3150800526813D001212046FFF769FF034668B9A169EB
S315080052783046FFF7B9FB034638B9E2691278E52ADA
S31508005288ECD0002AEAD00025EBE7042B01D0184613
S31508005298F8BD0723FBE72DE9F8430446884607685F
S315080052A84FF0FF094E4604252EE00F2B19D112F0B0
S315080052B8400F06D091F80D9002F0BF022369636289
S315080052C81646B24201D0FF2618E04B7B4B4501D063
S315080052D8FF2613E0A06AFFF73BFA88B3013EF6B249
S315080052E80CE026B90846FFF703FB48452BD04FF0D4
S315080052F8FF33636227E0FF2600E0FF2600212046E9
S31508005308FFF71CFF0546F0B9A169E1B13846FFF772
S315080053186BFB0546B8B9E1690A789AB1CB7A03F006
S315080053283F03A371E52AE6D02E2AE6D023F020000B
S31508005338082814BF002001204045B6D0FF26DDE71F
S31508005348FF26DBE704250DB10023A3612846BDE83F
S31508005358F88370B5044605680669416AB1F1FF3FE6
S3150800536818D1A1692846FFF73FFB034670B9E269D9
S31508005378E52111700122EA702269B24206D200219B
S315080053882046FFF7DBFE03460028EAD0042B07D0A1
S31508005398184670BDFFF759FD03460028E1D0F7E720
S315080053A80223F5E72DE9F04F83B080468A46D1F8FF
S315080053B80090856A002411E0013609EB060219F8FF
S315080053C806302F2BF8D05C2BF6D0CAF800201F28F9
S315080053D821D8042722E025F814703446661C19F8E3
S315080053E804001F28E9D92F28E7D05C28E5D0FE2C29
S315080053F800F2DF80012100F0E9FF0746002800F0E7
S31508005408DA807F28E7D801466D48FFF766F900284D
S31508005418E1D0062086E0002700E0013C44B104F10B
S315080054280043013B35F81330202BF6D02E2BF4D049
S31508005438002325F81430002C00F0BF800B22202109
S31508005448D8F82000FFF735F9002300E0013335F8CE
S315080054581320202AFAD02E2AF8D01BB147F00307C2
S3150800546800E0013C6CB104F10042013A35F812201B
S315080054782E2AF6D14FF0080B4FF0000ACDF804A0F3
S315080054880AE0A2464FF0080B0022019204E04C45B8
S315080054980BD047F003074B4603F1010935F81360AB
S315080054A8FEB1202EF5D02E2EF1D0DA4510D24C4575
S315080054B80ED07F2E46D8002E51D147F003075F2617
S315080054C8D8F8203003F80A604B460AF1010AE3E7E0
S315080054D8BBF10B0F29D04C4501D047F003074C45C3
S315080054E826D2D8F820301A78E52A54D0BBF1080F06
S315080054F854D0019B03F00C020C2A03D003F00303D3
S31508005508032B01D147F0020717F0020F06D1019BBA
S3150800551803F00303012B46D0042A47D0D8F82030D5
S31508005528DF72002003B0BDE8F08F47F00307D8E71D
S31508005538019B9B00DBB2019323464FF00B0B4FF000
S31508005548080AA9E70021304600F040FF064618B1C8
S31508005558A0F180061B4B9E5D47F00207ABE7314674
S315080055681948FFF7BAF80028A7D1A6F141039BB254
S31508005578192B04D8019B43F002030193A0E7A6F16F
S3150800558861039BB2192B9BD8019B43F00103019336
S31508005598203EB6B294E705221A70A7E7019B9B003E
S315080055A8DBB20193A5E747F01007B5E747F0080708
S315080055B8B4E70620B6E70620B4E70620B2E700BF38
S315080055C848690008B868000854690008F8B500234F
S315080055D88B758369002B6BD00D460646436AB3F173
S315080055E8FF3F13D0836A00249F1C188858B10021EE
S315080055F800F0ECFE30B1FE2C0CD82A1990753B4603
S315080056080134F1E700242C440023A375A87D002261
S31508005618134612E00024F6E7E52317E010B9A9189F
S315080056282E278F75A9182E274F72013210E01021E0
S315080056381CE0A9188B75013223460A2B1BD8F16979
S315080056485C1CCB5C202BF7D0052BE5D0092CE5D0C4
S31508005658A9184B720028EED1A3F14101C9B219293C
S31508005668E7D8F1690F7B082CE1D808210F42E0D06A
S315080056782033DBB2DDE730B9AB1800219975F36939
S315080056881B7B03B90A462A4400235372F369DB7A5B
S315080056982B72F0691C30FEF7EAFF2860F0691830AB
S315080056A8FEF7E0FFA880F0691630FEF7DBFFE88012
S315080056B8F8BD00002DE9F04781460F4601F11A00AA
S315080056C8FEF7D0FFB8BB3D7805F03F05013D05EB71
S315080056D8450305EB83054FF00108002404E04FF65F
S315080056E8FF7398422ED101340C2C18D8194B185D23
S315080056F83844FEF7B7FF0646B8F1000FEFD0FE2D7F
S315080057081CD800F07FFE804605F1010A39F8150015
S3150800571800F078FE804513D1B0465546E3E73B7856
S3150800572813F0400F10D0B8F1000F0FD039F8153024
S3150800573873B9012000E00020BDE8F0870020FBE7E8
S315080057480020F9E70020F7E70120F5E70120F3E74D
S315080057580020F1E7386900082DE9F8430446D0F82F
S3150800576800800021FFF771FB064600285ED14FF03E
S31508005778FF3363624FF0FF094F460AE04FF0FF33E5
S315080057886362FF2700212046FFF7D8FC0646002853
S315080057984CD1A1694046FFF727F90646002845D1A6
S315080057A8E5692B78002B40D0E97A01F03F02A2710F
S315080057B8E52BE3D011F0080F01D00F2ADED10F2A06
S315080057C814D027B92846FFF793F848452ED0216AFA
S315080057D8CB7A13F0010F04D10B222846FEF76EFF89
S315080057E820B34FF0FF336362FF27CBE7A06A002890
S315080057F8C8D013F0400F06D095F80D9003F0BF03F4
S31508005808226962621F46BB4201D0FF27BAE76B7B53
S315080058184B4501D0FF27B5E72946FFF74BFF10B1DF
S31508005828013FFFB2AEE7FF27ACE704263046BDE8DE
S31508005838F88330B583B004460191056801E0013361
S315080058480193019B1A782F2AF9D05C2AF7D00022EF
S31508005858A2601B781F2B1DD901A92046FFF7A2FDB8
S315080058680346F8B92046FFF777FF236ADA7A03462C
S31508005878D8B912F0040F15D1A37913F0100F1BD05D
S315080058882169C1F30801303129442846FEF739FF52
S31508005898A060E1E7236A8022DA7200212046FFF732
S315080058A8D4FA0346184603B030BD0428FAD112F0D4
S315080058B8040FF7D10523F5E70523F3E72DE9F047A4
S315080058C884B00668D0F820A0D0F828809AF80B305B
S315080058D813F0A00F40F08980002400E0013438F85E
S315080058E81430002BFAD105460C22514601A8FEF7BA
S315080058F8D7FE9DF80F3013F0010F1ED000238AF843
S315080059080B30AB620127632F0CD83B46424601A9E8
S315080059185046FEF79DFF2846FFF71EFF814608B941
S315080059280137F0E7642F66D0B9F1040F5FD19DF807
S315080059380F308AF80B30C5F828809DF80F3013F019
S31508005948020F2AD00C342D4BA3FB0434A4080134C7
S3150800595821462846FFF777FC814608B9013C1ED13F
S31508005968B9F1000F43D1A9693046FFF73DF88146DA
S3150800597800283CD120220021E869FEF79AFE0B226E
S31508005988296AE869FEF78CFE2B6ADB7AEA6903F06E
S31508005998180313730123F37029E00124D8E729694A
S315080059A8A1EB44112846FFF750FA81460028D7D1BB
S315080059B8286AFEF79DFF0746A9693046FFF714F8D7
S315080059C881460028CCD13B46E2B2E969A86AFEF7C7
S315080059D803FF0123F37000212846FFF7AFFB814632
S315080059E80028BDD1013CE7D1BAE74FF00609484679
S315080059F804B0BDE8F0874FF00709F8E74FECC44E46
S31508005A0870B50446FEF7C6FF054648B92378032B42
S31508005A1808D0002211466078FDF737FB00B101254A
S31508005A28284670BD2379012BF3D104F130064FF4CB
S31508005A38007200213046FEF73CFE4AF6552104F26C
S31508005A482E20FEF71FFE0F493046FEF71FFE0E49A9
S31508005A5804F50570FEF71AFE216904F50670FEF7C7
S31508005A6815FEE16804F50770FEF710FEE2690132D3
S31508005A78E262012331466078FDF702FB00232371B1
S31508005A88C7E700BF525261417272416110B584B0CE
S31508005A9801900091144604A840F8041DFEF736FF45
S31508005AA8002819DB0E4B53F820300BB100221A7068
S31508005AB8019B0BB100221A70019B094A42F8203053
S31508005AC863B1012C02D0002004B010BD002201A940
S31508005AD86846FEF7D3FFF7E70B20F5E70020F3E75C
S31508005AE8700F00202DE9F04393B00191002800F0CB
S31508005AF8AF80044615460023036002F01F073A469E
S31508005B0806A901A8FEF7BAFF064618B1304613B02B
S31508005B18BDE8F083069B079303AB0F934D4B119390
S31508005B28019907A8FFF785FE064620B90F9B93F942
S31508005B380B30002B46DB15F01C0F54D0002E48D02E
S31508005B48042E41D047F00807002E5BD117F0080F3E
S31508005B5858D0414D29460E980E30FEF797FD29462E
S31508005B680E981630FEF792FD0E9B2022DA72069DD5
S31508005B78DDF8388041462846FEF7C3FD81460022EF
S31508005B8841462846FEF7D0FD00210E981C30FEF740
S31508005B987DFD069B0122DA70B9F1000F32D0069B0B
S31508005BA8DD6A0022494607A8FFF789FA064648BB70
S31508005BB829460698FEF718FF064609F1FF33069A9E
S31508005BC8D3601FE00626B6E707A8FFF777FE06465E
S31508005BD8B8E79DF8223013F0110F12D115F0040F0B
S31508005BE8B2D008260EE06EB99DF8223013F0100FD1
S31508005BF82CD115F0020F05D013F0010F02D0072695
S31508005C080BE007264EB917F0080F01D047F0200712
S31508005C18069BDB6A23620E9B6362002E7FF476AFCF
S31508005C28069DDDF8388041462846FEF76AFDA060DD
S31508005C3808F11C00FEF71BFDE0600023637463612E
S31508005C48E36127742560EB88A3805FE70426E4E709
S31508005C5809265BE7780F0020000061482DE9F04F18
S31508005C6885B004468946174698460023C8F8003082
S31508005C7803A9FEF775FE0646002840F0A280667C52
S31508005C88002E40F09E80237C13F0010F00F0A380BD
S31508005C98E5686369ED1ABD425DD33D465BE0A169D7
S31508005CA82046FFF76BF866E00226667489E0012647
S31508005CB8667486E00226667483E0237C13F0400F38
S31508005CC805D0E069A0EB0A00019B984202D3019B24
S31508005CD85F0236E04FF4007204F1280109EB402010
S31508005CE8FEF7DEFCF3E7E26952451AD0237C13F087
S31508005CF8400F0CD0012304F128019BF80100FDF799
S31508005D08BFF9002861D1237C23F0400323740123BB
S31508005D18524604F1280103984078FDF7ACF90028A3
S31508005D2856D1C4F81CA06169C1F30801C1F500770A
S31508005D38BD4200D22F4628313A4621444846FEF746
S31508005D48AFFCB94463693B446361D8F800303B4407
S31508005D58C8F80030ED1B002D33D06369C3F3080279
S31508005D68002AE0D1039A5789013F17EA532708D131
S31508005D78002B94D1A068012896D9B0F1FF3F96D098
S31508005D88A061DDF80CB0A1695846FEF7AEFC82465C
S31508005D9800288FD0BA446B0A0193A4D0FB18BBF825
S31508005DA80A20934201D9D31B0193019B52464946BF
S31508005DB89BF80100FDF75FF900283FF47EAF01263E
S31508005DC86674304605B0BDE8F08F01266674F8E7B4
S31508005DD801266674F5E70726F3E72DE9F04F85B03F
S31508005DE804468846154699460023C9F8003003A98B
S31508005DF8FEF7B6FD0746002840F0B280677C002FFC
S31508005E0840F0AE80237C13F0020F00F0BF80636970
S31508005E18EB4264D3DD4362E000212046FFF7EDF844
S31508005E286FE0A1692046FFF7E8F86AE00227677479
S31508005E3896E00127677493E00123E26904F12801D3
S31508005E4803984078FDF71CF920B9237C23F0400312
S31508005E58237465E00127677482E0022767747FE088
S31508005E68E169A1EB0A01594502D34FEA4B2627E017
S31508005E784FF4007208EB412104F12800FEF710FCE4
S31508005E88237C23F040032374EFE7E369534503D0E3
S31508005E986269E3689A4267D3C4F81CA06069C0F3CC
S31508005EA80800C0F50076B54200D22E46283032469C
S31508005EB841462044FEF7F4FB237C43F04003237451
S31508005EC8B044636933446361E268934238BF134652
S31508005ED8E360D9F800303344C9F80030AD1B002D0B
S31508005EE84FD06369C3F30802002AD7D1039A5689A3
S31508005EF8013E16EA53260FD1002B92D1A068002836
S31508005F088AD000283DD0012890D0B0F1FF3F90D024
S31508005F18A061A36803B9A060237C13F0400F8BD156
S31508005F28039B0193A1691846FEF7DFFB8246002802
S31508005F3893D0B2445FEA552BA7D006EB0B03019A18
S31508005F485289934201D9A2EB060B5B465246414653
S31508005F5801984078FDF794F8002881D001276774DE
S31508005F68384605B0BDE8F08F0123524604F12801EA
S31508005F7801984078FDF77FF800288DD001276774C7
S31508005F88EEE7237C43F020032374E9E70727E7E7CE
S31508005F9870B582B004460D460A290DD06368002BF1
S31508005FA808DB5E1C23441D733C2E09DC6660A36867
S31508005FB80133A36002B070BD0D21FFF7E9FFEDE7D5
S31508005FC801AB324604F10C012068FFF706FF019B76
S31508005FD89E4202D04FF0FF36E8E70026E6E70000C3
S31508005FE830B583B0044601A9FEF7BAFC0346C8B91A
S31508005FF8227C12F0200F15D012F0400F0CD0012386
S31508006008E26904F1280101984078FDF739F888BB58
S31508006018237C23F040032374216A0198FEF7E4FCE5
S31508006028034610B1184603B030BD656AEB7A43F0EB
S315080060382003EB72A26829462068FEF775FBE1681B
S3150800604805F11C00FEF722FB0B4905F11600FEF7C1
S315080060581DFB002105F11200FEF714FB019B012226
S31508006068DA700198FFF7CCFC0346227C22F020025E
S315080060782274D7E70123D5E70000614810B582B036
S315080060880446FFF7ADFF034610B1184602B010BD27
S3150800609801A92046FEF764FC03460028F5D100222C
S315080060A82260F2E72DE9F04182B004460F4601A9BD
S315080060B8FEF756FC0646002840F0A280667C002EAD
S315080060C840F09E80E368BB4204D2227C12F0020F9D
S315080060D800D11F46636900226261002F65D0019AC4
S315080060E8B2F80A804FEA482873B17A1EB2FBF8F26A
S315080060F8013BB3FBF8F18A4206D3C8F10002134004
S315080061086361FF1AA56902E0A56815B1A56135BBE3
S315080061184CE000212046FEF770FF0546012804D00A
S31508006128B0F1FF3F04D0A060F0E70226667467E086
S315080061380126667464E029462046FEF71FFE0546D2
S31508006148B5F1FF3F28D0012D29D9019B5B69AB42E0
S3150800615825D9A561636943446361A7EB08074745E1
S315080061680BD9237C13F0020FE5D029462046FEF703
S3150800617844FF05460028E3D1474663693B44636103
S31508006188C7F30803002B3FD029460198FEF7ADFA56
S3150800619840B100EB572509E00126667430E002266F
S315080061A866742DE0022666742AE000256369C3F33F
S315080061B80803E3B1E269AA4219D0237C13F0400F19
S315080061C80BD0012304F1280101984078FCF758FF01
S315080061D8E0B9237C23F04003237401232A4604F1FB
S315080061E8280101984078FCF746FF90B9E56163698C
S315080061F8E268934204D9E360237C43F020032374BE
S31508006208304602B0BDE8F0810025CFE7012666745E
S31508006218F6E701266674F3E730B591B001900D46A6
S31508006228002205A901A8FEF729FC044610B1204654
S3150800623811B030BD02AB0D930B4B0F93019905A80E
S31508006248FFF7F7FA04460028F1D10D9B93F90B30AE
S31508006258002B06DB002DEAD0294605A8FFF7B6F974
S31508006268E5E70624E3E700BF780F0020F0B59DB000
S315080062780190022205A901A8FEF700FC059B1193C7
S31508006288044610B120461DB0F0BD02AB1993254B44
S315080062981B93019911A8FFF7CCFA04460028F1D1F7
S315080062A8199B93F90B30002B1EDB9DF84A5015F005
S315080062B8010F2AD1059F18993846FEF722FA06468D
S315080062C815F0100F12D006970890002106A8FEF7B9
S315080062D8BCFD044650B9002106A8FEF7DCFF0446B3
S315080062E8B0B1042802D103E000260624002CC9D13F
S315080062F811A8FFF72EF8044600B95EB9002CC1D1DB
S315080063080598FFF77DFB0446BCE700260724EDE75A
S315080063180724EBE70022314611A8FEF7D0FE04460B
S31508006328ECE700BF780F00202DE9F04182B08046DF
S315080063380E4617460446002501E022461446731EF3
S31508006348AB4212DD6B46012201A93846FFF786FCE7
S31508006358009B012B09D19DF804300D2BEDD0621C4A
S31508006368237001350A2BE9D11446002323701DB181
S31508006378404602B0BDE8F0810020FAE710B594B0AF
S315080063880446019100230293039303E0013401A80C
S31508006398FFF7FEFD21780029F8D1029A002A0CDBBE
S315080063A86B4604A90198FFF718FD48B9029A009B9D
S315080063B89A4208D1039814B010BD4FF0FF30FAE797
S315080063C84FF0FF30F7E74FF0FF30F4E77F2816D98C
S315080063D831B1FF2812D88038094B33F810007047B6
S315080063E800237F2B07D8064A32F81320824202D0A8
S315080063F801339BB2F5E78033D8B27047002070475F
S315080064085C690008B0F5805F07D2234B1A88002A12
S3150800641840D090423ED3F0B406E0204BF6E72B4630
S315080064281A88CAB1904217D31D1D5B88190ADBB2B0
S315080064389C18A04204DB0029F1D105EB4303EFE7DA
S31508006448082909D8DFE801F0050A101316191C1FD0
S315080064582200861A35F81600F0BC7047821A02F030
S315080064680103C01A80B2F7E7103880B2F4E720387B
S3150800647880B2F1E7303880B2EEE71A3880B2EBE737
S31508006488083080B2E8E7503880B2E5E7A0F5E3506F
S3150800649880B2E1E7704700BF5C6A0008506C0008E4
S315080064A870B50D4E0D4CA41BA4100025A54209D1A4
S315080064B80B4E0C4C00F04EF8A41BA4100025A54260
S315080064C805D170BD56F8253098470135EEE756F8D8
S315080064D8253098470135F2E7206E0008206E000837
S315080064E8206E0008246E0008044B054A1B681B6AC0
S315080064F8002B08BF1346D3F8EC007047100000209D
S315080065087400002082B001B901A942B14BB11378D1
S315080065180B601278101C18BF012002B0704710468D
S31508006528FBE76FF00100F8E702440346934200D1FF
S31508006538704703F8011BF9E749B1FF2A85BF8A2383
S3150800654803600A704FF0FF3098BF0120704708466D
S3150800655870470000F8B500BFF8BC08BC9E467047EF
S31108006568F8B500BFF8BC08BC9E4670479A
S315080065742F626F6F746C6F672E7478740000000056
S315080065842F64656D6F70726F675F6F6C696D657880
S315080065945F73746D3332653430372E7372656300F6
S315080065A400000000000000000102030406070809B1
S315080065B40000000001020304433A2F576F726B2F41
S315080065C4736F6674776172652F4F70656E424C54AB
S315080065D42F5461726765742F536F757263652F4103
S315080065E4524D434D345F53544D333246342F636111
S315080065F46E2E630005020602060307030803090351
S3150800660409040A040B040C040C050D050E050F05F4
S315080066140F06100610071008008000080040000046
S315080066240200000000C0000800400000030000004B
S315080066340000010800000100040000000000020830
S315080066440000020005000000000004080000020023
S31508006654060000000000060800000200070000000B
S3150800666400000808000002000800000000000A08EC
S31508006674000002000900000000000C0800000200E7
S315080066840A00000000000E08000002000B000000CB
S31508006694433A2F576F726B2F736F667477617265FF
S315080066A42F4F70656E424C542F5461726765742F70
S315080066B4536F757263652F41524D434D345F53547E
S315080066C44D333246342F72733233322E6300000050
S315080066D4303A0000433A2F576F726B2F736F667404
S315080066E4776172652F4F70656E424C542F546172F0
S315080066F46765742F536F757263652F66696C652EAB
S31508006704630000004669726D77617265207570646E
S315080067146174652072657175657374206465746542
S31508006724637465640A0D00004F70656E696E6720B0
S315080067346669726D776172652066696C6520666F35
S31508006744722072656164696E672E2E2E0000000041
S315080067544552524F520A0D004F4B0A0D00000000D5
S315080067645374617274696E67207468652070726FF9
S315080067746772616D6D696E672073657175656E63A1
S31508006784650A0D0050617273696E67206669726DD9
S31508006794776172652066696C6520746F2064657418
S315080067A465637420657261736520626C6F636B73CD
S315080067B42E2E2E0045726173696E67200000000054
S315080067C42062797465732066726F6D206D656D6FCE
S315080067D47279206174203078000000005265616483
S315080067E4696E67206C696E652066726F6D206669CE
S315080067F46C652E2E2E4552524F520A0D000000008B
S31508006804496E76616C696420636865636B73756D3C
S3150800681420666F756E642E2E2E4552524F520A0DFF
S315080068240000000050726F6772616D6D696E6720B3
S315080068340000000020627974657320746F206D650A
S315080068446D6F72792061742030780000577269740C
S31508006854696E672070726F6772616D20636865631D
S315080068646B73756D2E2E2E00436C6F73696E6720DD
S315080068746669726D776172652066696C650A0D00D2
S315080068844669726D776172652075706461746520F6
S315080068947375636365737366756C6C7920636F6D62
S315080068A4706C657465640A0D000000004F70656EAF
S315080068B4424C5400809A45418E418F80454545494E
S315080068C449498E8F9092924F994F555559999A9B4B
S315080068D49C9D9E9F41494F55A5A5A6A7A8A9AAABC5
S315080068E4ACADAEAFB0B1B2B3B4B5B6B7B8B9BABB5E
S315080068F4BCBDBEBFC0C1C2C3C4C5C6C7C8C9CACB4E
S31508006904CCCDCECFD0D1D2D3D4D5D6D7D8D9DADB3D
S31508006914DCDDDEDFE0E1E2E3E4E5E6E7E8E9EAEB2D
S31508006924ECEDEEEFF0F1F2F3F4F5F6F7F8F9FAFB1D
S31508006934FCFDFEFF01030507090E10121416181CA8
S315080069441E000000222A3A3C3E3F7C7F00000000DD
S315080069542B2C3B3D5B5D0000C700FC00E900E20010
S31508006964E400E000E500E700EA00EB00E800EF00D9
S31508006974EE00EC00C400C500C900E600C600F40039
S31508006984F600F200FB00F900FF00D600DC00A200C6
S31508006994A300A500A7209201E100ED00F300FA0088
S315080069A4F100D100AA00BA00BF001023AC00BD0054
S315080069B4BC00A100AB00BB009125922593250225B6
S315080069C424256125622556255525632551255725F0
S315080069D45D255C255B251025142534252C251C25C9
S315080069E400253C255E255F255A25542569256625F7
S315080069F4602550256C256725682564256525592550
S31508006A045825522553256B256A2518250C258825CE
S31508006A1484258C2590258025B103DF009303C003C4
S31508006A24A303C303B500C403A6039803A903B403C5
S31508006A341E22C603B50329226122B10065226422F7
S31508006A4420232123F7004822B0001922B7001A226E
S31508006A547F20B200A025A00061001A03E0001703F6
S31508006A64F8000703FF000100780100013001320134
S31508006A740601390110014A012E0179010601800136
S31508006A844D00430281018201820184018401860149
S31508006A948701870189018A018B018B018D018E018A
S31508006AA48F0190019101910193019401F6019601D8
S31508006AB49701980198013D029B019C019D012002C2
S31508006AC49F01A001A001A201A201A401A401A6019B
S31508006AD4A701A701A901AA01AB01AC01AC01AE014A
S31508006AE4AF01AF01B101B201B301B301B501B501FB
S31508006AF4B701B801B801BA01BB01BC01BC01BE01AA
S31508006B04F701C001C101C201C301C401C501C40121
S31508006B14C701C801C701CA01CB01CA01CD011001C9
S31508006B24DD0101008E01DE011201F3010300F1010A
S31508006B34F401F401F8012801220212013A020900BB
S31508006B44652C3B023B023D02662C3F024002410291
S31508006B54410246020A015302400081018601550298
S31508006B6489018A0158028F015A0290015C025D026A
S31508006B745E025F0293016102620294016402650285
S31508006B8466026702970196016A02622C6C026D021C
S31508006B946E029C01700271029D01730274029F01C8
S31508006BA476027702780279027A027B027C02642CE6
S31508006BB47E027F02A60181028202A901840285025D
S31508006BC486028702AE014402B101B20145028D0272
S31508006BD48E028F0290029102B7017B030300FD0324
S31508006BE4FE03FF03AC0304008603880389038A03B0
S31508006BF4B1031103C2030200A303A303C4030803D6
S31508006C04CC0303008C038E038F03D8031801F20305
S31508006C140A00F903F303F403F503F603F703F7038A
S31508006C24F903FA03FA033004200350041007600436
S31508006C3422018A043601C1040E01CF040100C004EE
S31508006C44D004440161052604000000007D1D0100EE
S31508006C54632C001E9601A01E5A01001F0806101F69
S31508006C640606201F0806301F0806401F0606511F81
S31508006C740700591F521F5B1F541F5D1F561F5F1FB6
S31508006C84601F0806701F0E00BA1FBB1FC81FC91F46
S31508006C94CA1FCB1FDA1FDB1FF81FF91FEA1FEB1FDA
S31508006CA4FA1FFB1F801F0806901F0806A01F080668
S31508006CB4B01F0400B81FB91FB21FBC1FCC1F0100A8
S31508006CC4C31FD01F0206E01F0206E51F0100EC1FC2
S31508006CD4F21F0100FC1F4E2101003221702110020F
S31508006CE4842101008321D0241A05302C2F04602C1A
S31508006CF40201672C0601752C0201802C6401002D03
S31508006D04260841FF1A0300004300504F5349580010
S31508006D142E00002020202020202020202828282873
S31508006D242820202020202020202020202020202049
S31508006D342020208810101010101010101010101099
S31508006D4410101004040404040404040404101010A9
S31508006D541010101041414141414101010101010155
S31508006D6401010101010101010101010101011010E3
S31508006D741010101042424242424202020202020229
S31508006D8402020202020202020202020202021010B5
S31508006D9410102000000000000000000000000000A1
S31508006DA400000000000000000000000000000000D1
S31508006DB400000000000000000000000000000000C1
S31508006DC400000000000000000000000000000000B1
S31508006DD400000000000000000000000000000000A1
S31508006DE40000000000000000000000000000000091
S31508006DF40000000000000000000000000000000081
S31508006E040000000000000000000000000000000070
S30908006E14000000006C
S30D08006E18E093FF7F0100000072
S30908006E20AD010008AA
S30908006E2489010008CA
S31508006E280024F4000100000010000000010400001E
S31508006E381400002000000000000000000000000008
S31508006E48000000000000000000000000000000002C
S31508006E58000000000000000000000000000000001C
S31508006E68000000000000000000000000000000000C
S31508006E7800000000000000000000000000000000FC
S31508006E8800000000000000000000000000000000EC
S31508006E980000000043000000000000000000000099
S31508006EA800000000000000000000000000000000CC
S31508006EB80000000043000000000000000000000079
S31508006EC800000000000000000000000000000000AC
S31508006ED80000000043000000000000000000000059
S31508006EE8000000000000000000000000000000008C
S31508006EF80000000043000000000000000000000039
S31508006F08000000000000000000000000000000006B
S31508006F180000000043000000000000000000000018
S31508006F28000000000000000000000000000000004B
S31508006F3800000000430000000000000000000000F8
S31508006F48000000000000000000000000000000002B
S31508006F5800000000430000000000000000000000D8
S31508006F68000000000000000000000000000000000B
S31508006F7800000000416500080D65000800000000D3
S31508006F88166D0008146D0008156D0008156D0008C3
S31508006F98156D0008156D0008156D0008156D0008B3
S31508006FA8156D0008156D0008156D0008FFFFFFFF31
S31508006FB8FFFFFFFFFFFFFFFFFFFF00000100415330
S31508006FC843494900000000000000000000000000D6
S31508006FD80000000000000000000000000000415307
S31508006FE843494900000000000000000000000000B6
S31508006FF8000000000000000000000000000000007B
S70508000AD513
